:100000000C94EC0C0C94140D0C94140D0C94140D15
:100010000C94140D0C94140D0C94140D0C94140DDC
:100020000C94140D0C94140D0C94AF1D0C941E1E06
:100030000C94140D0C94140D0C94140D0C94140DBC
:100040000C94140D0C94140D0C94140D0C94140DAC
:100050000C94140D0C94140D0C94140D0C9450204D
:100060000C94140D0C94140D0C94140D0C94140D8C
:100070000C94140D0C94140D0C94140D0C94140D7C
:100080000C949A200C94140D0C94140D0C94140DD3
:100090000C94140D0C94140D0C94140D0C94140D5C
:1000A0000C94140D0C94140D0C94140D1818BB0E14
:1000B0000C0A03150A0A020A040A1002090E020BAE
:1000C0000C03070D04030E05030E0A030F0C030FA8
:1000D0000D030C12032312021015030E0A000C0B61
:1000E000000C0D000C07010F06010D0C080E130685
:1000F0001011060F0C060D0411100611080B0F0944
:100100000C0F090D0F090F03110D0D11130B0F1516
:100110000B0D140A0C0C140E0D160D0A150D0915F5
:100120000F07130C06130E02150F00140C03130E09
:100130001012080F140E15170216170210172311AC
:100140001723121723131723141723171422171515
:10015000221716221717221115221116220F170720
:100160000E17200D17200C17200B16200B17200A36
:1001700016200A1720091620091720081420081530
:10018000200816200817200714200715200716201E
:10019000071720061520061620061720051620052D
:1001A000172004160704172003160703172002164A
:1001B000200217200114200115200116200117200C
:1001C00000152000162000172013122314122315E7
:1001D00012230C13230D13230E13230F13231013B9
:1001E000230E14220E1522021223031223041223BB
:1001F00005122306122307122308122307102207D1
:100200001122020C22020D22020E22020F220210E3
:10021000220B0E230C0E230D0E230C0C220C0D2290
:10022000100B22100C22100D22100E22110E231280
:100230000E23130E23140E23150E23160E23170E52
:1002400023140B20130C20140C20150C20140D0368
:10025000160923170923040B23050B23060B230080
:100260000A231007231107231207231307230C0760
:100270002306050308082302082303082305062391
:100280000606230706230806230805220804230977
:1002900004230A04230B04230C04230D0423140257
:1002A000231502230801230901230A01230B01233B
:1002B0000C01230D01230E01230F01231001230440
:1002C0000223050223060223070223000223010260
:1002D000230001050E03230F032310032312160C22
:1002E00018189812042004160D0B120E04100E0E8E
:1002F0000D0F0A0D0F0B0D0D0D0D0D120B0C0C0932
:100300000E0D090E0B090E0C030D020A0C04171832
:100310000917190B17180E17190A1603130E030ADB
:10032000100305010A0C020A13030A0C060B12162D
:100330000816170215170201170202170217171BDA
:1003400014171800171B031719131017131117137D
:100350001217131317131417131517131617130F58
:1003600016161319161409140F18120F1912100962
:10037000141009100D09110D09120D09130D09149E
:100380000D09150D09160D09100C16110C16120C7D
:1003900016130C16140C16150C16160C160F0C1E34
:1003A0000F0D170F0E170F0F170F10170F11170F35
:1003B00012170F13170F141D1013181014090E1411
:1003C000190E11190B11210B14210C17080D170808
:1003D0000517070617070717070817070114210253
:1003E00014210314210414210514210614210714D7
:1003F000210814210914210A1421011307021307EB
:100400000313070413070513070613070713070849
:1004100013070911210A11210912210A12210913B6
:10042000210A1321040F20090E200A0E200B0E2092
:100430000C0E200D0E200E0E20090B20090C200999
:100440000D20060920060A20060B20070B20080BAA
:1004500020010B20020B20030B20010A200308209F
:100460000408200508200608200708200908200A9B
:1004700008200B08200C08200D08200E08200F086B
:100480002010082011082012082013082015082029
:100490001608200B0B210C0B210D0B210504200647
:1004A00004200B04200C0420110420120420041743
:1004B0001818061C0D040D0C040F0B040D00001A77
:1004C000030019010321010421040121040421175F
:1004D000020217030217011B17041A01000202008F
:1004E0000210042111042112042113042109032103
:1004F0000A03210B03210C03210D03211203030C1A
:1005000002030D04030C010A0C060E060322060466
:10051000220703110A040C01040F02040D09010E45
:1005200005010E02000203000205020A0805020985
:1005300005020203201818B4160E0E01050E0A0E4D
:100540000C070E01060E0A14000215000213001813
:1005500016001900020200030200011B00041E1213
:1005600003161303161403161503161603160A03AF
:100570001A0B03070C03070D031E0E031C0F0307C2
:1005800010030711031E0A041F0B04160C04160D9A
:1005900004160E04160F0416100416110416120485
:1005A0001D07011707021707031707041707051789
:1005B00007061707071F0807160907160A07160B6D
:1005C00007160C07160D07160E07160F071610074D
:1005D0001611071612071613071614071D14061A0C
:1005E0000A0603160A1E150A08140A08130A080F39
:1005F0000809100809110809120A1C110A16100A24
:10060000160F0A1E0C08170C09170C0A170C0B17EB
:100610000C0C170C0D170C0E170C0F170C10170CD9
:1006200011170C12170C13170F0B170F0C170F0DB8
:10063000170F0E170F0F170F10170E0D080E0E19AC
:100640000D11080D1218120D16130D16140D161596
:100650000D16160D16110D1E110E17110F17111074
:100660001711111D1011160F111F120B1F130B164E
:10067000140B16150B16160B1614101A141117144A
:10068000121714131714141D0D14160E14160F142C
:10069000161014161114161214161314160C141F17
:1006A00016160715161A11161A1315090F1509092A
:1006B0000D17090E17090F1F0A0F160B0F16091039
:1006C0000909141A0915170916170615160715161C
:1006D000081516070F1505121A0513170514170527
:1006E0001517051617040C16050C16060C16070C24
:1006F00016080C16090C160A0C160B0C16030C1E09
:10070000050D0903141D02141901101804161E0307
:10071000160702161A030D17030E17030F170310FF
:1007200017031117031217031317010418040318F2
:10073000030319040409030409040718030719042F
:100740000809030809070A19080A16090A180714EC
:1007500003070B0306181C020C0E02000203000222
:100760000100180400190202190302180106080109
:100770000718040719010A08020A08030A08010BEE
:1007800016020B16030B18040E19011108031108A9
:100790000112180312150215150116080416080196
:1007A00017180417190217020317020C0C2E06095A
:1007B0000E09010E04020D07060C04060306010AC9
:1007C0000A0204000900000A02030B08040B0801D6
:1007D0000820020820030809040809050820060863
:1007E000200708200808200A09200A0A20010720FB
:1007F000020720030720040720050720060720071B
:1008000007200905090A050903042004042005043A
:10081000200604200704200804200904200A0420DC
:100820000403200803200903200A032002052005F1
:1008300003070603070703070C0C2D08060E07081D
:100840000C04030D0A060F0A010A0200020300004D
:10085000020B02030B020B02000B03000B0302004E
:100860000B1F010B18040B19050B1D0007170008BF
:1008700017000917000A1700061E010616020616C1
:1008800003061604061605061C05071B050A1A06AC
:100890000B07070B07080B07090B070A0B070709CC
:1008A000200A072008052004042005042004052050
:1008B00005052002022008022001050702050703A2
:1008C00005070C0C1E06020F01060D03050A0200A7
:1008D000180500190B01000B02020B00180B031C7A
:1008E0000A03190805180A07190809180701170744
:1008F0000217070317070417070517070617070747
:100900001707081707091F0107160207180503191B
:10091000060316030002040002020A200209061858
:10092000062916020E00021B00051904040705041F
:10093000070903070A03070E01090F010900030055
:1009400000040203041A0604190704160804160812
:10095000031A0904160A04160A05160B04160C04D9
:10096000180B031A0D05180E05020F0502100519C4
:10097000110419120416130416140416150416167D
:10098000041612011F13011D13001C12030316008D
:100990001E16011F1502151400021500020C0C1B77
:1009A0000A060D0304190404180704150B01000BB3
:1009B00002020B031A0B001800081B000B190A0592
:1009C000190907210A072107081A0908210A08211D
:1009D00007091F0809160909160A0916060A190740
:1009E0000A16080A16090A160A0A16000900000A59
:1009F00002F0F89C8E8783878E9CF8F00000FEFF43
:100A00000303030303070EFCF80000FEFF030303C8
:100A10000303070EFCF80000FFFF000000000000C9
:100A200000FFFF0000FEFF8383838383C7EE7C38D3
:100A30000000F8FC0E07030303070EFCF800003F5C
:100A40007FE0C08080C0E07F3FFFFF010101010126
:100A50000101FFFF0000FFFF0C0C0C0C1C3E77E3B4
:100A6000C100007FFFC0C0C0C0C0E0703F1F0000D9
:100A70001F3F70E0C0C0C0E0703F1F00007FFFC19B
:100A8000C1C1C1C1E3773E1C00001F3F70E0C0C080
:100A9000C0E0703F1F000000000001FFFF010000E8
:100AA00000D5F08D14A1C881CFD9F1AF2000F40199
:100AB0003200900132002C016400F4011900900111
:100AC0001900008000000000003E5B4F5B3E3E6B63
:100AD0004F6B3E1C3E7C3E1C183C7E3C181C577DD8
:100AE000571C1C5E7F5E1C00183C1800FFE7C3E724
:100AF000FF0018241800FFE7DBE7FF30483A060E36
:100B00002629792926407F050507407F05253F5A7C
:100B10003CE73C5A7F3E1C1C08081C1C3E7F1422EC
:100B20007F22145F5F005F5F06097F017F00668997
:100B3000956A606060606094A2FFA29408047E04DD
:100B40000810207E201008082A1C08081C2A080803
:100B50001E101010100C1E0C1E0C30383E383006C3
:100B60000E3E0E06000000000000005F00000007BF
:100B7000000700147F147F14242A7F2A12231308ED
:100B8000646236495620500008070300001C2241C9
:100B9000000041221C002A1C7F1C2A08083E08086D
:100BA000008070300008080808080000606000201D
:100BB000100804023E5149453E00427F4000724900
:100BC0004949462141494D331814127F10274545A4
:100BD00045393C4A494931412111090736494949BA
:100BE00036464949291E0000140000004034000028
:100BF0000008142241141414141400412214080291
:100C0000015909063E415D594E7C1211127C7F4903
:100C10004949363E414141227F4141413E7F494958
:100C200049417F090909013E414151737F08080884
:100C30007F00417F41002040413F017F0814224155
:100C40007F404040407F021C027F7F0408107F3EAF
:100C50004141413E7F090909063E4151215E7F091C
:100C6000192946264949493203017F01033F404083
:100C7000403F1F2040201F3F4038403F631408146E
:100C80006303047804036159494D43007F414141A6
:100C90000204081020004141417F04020102044087
:100CA00040404040000307080020545478407F280B
:100CB0004444383844444428384444287F38545401
:100CC000541800087E090218A4A49C787F08040424
:100CD0007800447D40002040403D007F10284400C3
:100CE00000417F40007C047804787C080404783854
:100CF00044444438FC1824241818242418FC7C0884
:100D0000040408485454542404043F44243C404000
:100D1000207C1C2040201C3C4030403C44281028B3
:100D2000444C9090907C4464544C440008364100FC
:100D30000000770000004136080002010204023C76
:100D40002623263C1EA1A161123A4040207A385445
:100D500054555921555579412154547841215554C0
:100D6000784020545579400C1E5272123955555511
:100D700059395454545939555454580000457C41FC
:100D80000002457D420001457C40F0292429F0F015
:100D9000282528F07C545545002054547C547C0A66
:100DA000097F4932494949323248484832324A4833
:100DB00048303A4141217A3A42402078009DA0A033
:100DC0007D39444444393D4040403D3C24FF242487
:100DD000487E4943662B2FFC2F2BFF0929F620C0A4
:100DE000887E090320545479410000447D413048F5
:100DF000484A32384040227A007A0A0A727D0D1938
:100E0000317D2629292F28262929292630484D4099
:100E100020380808080808080808382F10C8ACBA95
:100E20002F102834FA00007B000008142A14222214
:100E3000142A14089500220095AA005500AAAA5564
:100E4000AA55AA000000FF00101010FF001414148F
:100E5000FF001010FF00FF1010F010F0141414FC2D
:100E6000001414F700FF0000FF00FF1414F404FC4A
:100E7000141417101F10101F101F1414141F00102B
:100E80001010F0000000001F101010101F101010A4
:100E900010F010000000FF101010101010101010B3
:100EA000FF10000000FF140000FF00FF00001F10F3
:100EB000170000FC04F414141710171414F404F4AD
:100EC0000000FF00F714141414141414F700F7149E
:100ED0001414171410101F101F141414F4141010ED
:100EE000F010F000001F101F0000001F1400000091
:100EF000FC140000F010F01010FF10FF141414FF89
:100F0000141010101F00000000F010FFFFFFFFFF83
:100F1000F0F0F0F0F0FFFFFF0000000000FFFF0F17
:100F20000F0F0F0F38444438447C2A2A3E147E02A7
:100F3000020606027E027E0263554941633844443C
:100F40003C04407E201E2006027E020299A5E7A5F1
:100F5000991C2A492A1C4C7201724C304A4D4D3062
:100F60003048784830BC625A463D3E494949007E87
:100F70000101017E2A2A2A2A2A44445F444440511E
:100F80004A444040444A51400000FF0103E080FFD2
:100F9000000008086B6B083612362436060F090F5E
:100FA00006000018180000001010003040FF01017A
:100FB000001F01011E00191D1712003C3C3C3C00A3
:100FC0000000000000B00000A170E150964F269094
:100FD0000F1D070C009669004AE44A00484440008F
:100FE000806810000F99FB8F9DBDBBFB77D4D4DFC9
:100FF0001F1A1AFE7F5D5DFF805A0000A0A4AA00A0
:1010000010BA3400FF5953F3FF9B9B9EFFB9B9966A
:10101000FF9595D19FF4940FFC295F91FF1838F844
:10102000FF9294FFFF95D5F7BFB5DDD7F18F81F122
:10103000F788C8F779C6467909FD9B090196F8003B
:101040008281828050716200775656007676370032
:10105000A2B773010772060078275000733474003A
:10106000775176007F55F7004771100032477200C4
:101070007364730015A2750061679400009F60603F
:10108000F4F2F6F20A050C1E1E1F1E1D1E1D1E0F79
:101090000C1E1F1E1D1E1D1E1F0C060F1E1D1E0DCD
:1010A0000E1F1E0C100A70F8CCCEFECFCFFD7F3F76
:1010B000EBFE76DCF8E0000000020202020202030E
:1010C00003030303010008073F7E7D7E7D7E7F3F93
:1010D0000A050F1E1D1E1D1E1F1E1E0C0C1F1E1D91
:1010E0001E1D1E1F1E0C0C1E1F0E0D1E1D1E0F068C
:1010F000100AE0F8DC76FEEB3F7FFDCFCFFECECCD2
:10110000F87000010303030303020202020202005B
:10111000000010080D0D191565A7A5470302629E72
:1011200066040C18081002050505025CE0000103C6
:10113000060AD4F72BFC1010C0F0B8F4FEFEFFFF37
:10114000FDFFFBEEFEF458E000010101E1F9F5E9D5
:10115000F5E9F5F9E10101000A10207F2000FF8088
:10116000FF840F0400000040FF4001000000002742
:1011700078208FFE050E05000000000040FF4000B3
:10118000000000277820FF009FE48F04000000404B
:10119000FF400001000010080C0A1DDFDFDF1B4EBE
:1011A000EC4000CC2C14B8300710E01806010618EB
:1011B000E0234489FE894423C0300C020C30C04730
:1011C0004892FC924827C0300C020C30C02748924D
:1011D000FC9248473FFFFFFFFFFF3F003FFFFFFF3D
:1011E000FFFF3F0000073FFF3F07000000073FFFF2
:1011F0003F07000010103FFFFF0000C03F003FFF0F
:10120000FF0000C03F0000073FC038070000000794
:101210003FC03807000000E0FCFFFCE0000000E0F9
:10122000FCFFFCE00000FCFFFFFFFFFFFC00FCFFF9
:10123000FFFFFFFFFC00101000E0FC031CE00000BB
:1012400000E0FC031CE00000FCFFFF000003FC00CA
:10125000FCFFFF000003FC00101001828204040464
:1012600002220102020404040202430404030000F7
:1012700000140060909060000100C42424C40402A3
:101280000282020202040404240488414180000016
:10129000000200060909060000001C24261A0302A9
:1012A000022C04629292610204040C12120C0000DF
:1012B00000A000000000000020001010FC02090D3A
:1012C0000D0D0D0D0D0D0D0D1D3902FC3F409AB495
:1012D000A8B0A8B0A8B0A8B0A890403F0D0D0D0DC3
:1012E0000D0D0D0D0D0D0D0D0D0D0D0DA8B0A8B0B2
:1012F000A8B0A8B0A8B0A8B0A8B0A8B0FF00AA55E0
:101300000000000000000000FFFF00FFFF00AA55E2
:101310000000000000000000FFFF00FF0D0D0D0D9C
:101320000D0D0D0D0D0D0D0D1D3902FCA8B0A8B051
:10133000A8B0A8B0A8B0A8B0A890403FFC02090D82
:101340000D0D0D0D0D0D0D0D0D0D0D0D3F409AB434
:10135000A8B0A8B0A8B0A8B0A8B0A8B0FC02A94D89
:101360000D0D0D0D0D0D0D1DFDF902FCFF00AA5513
:101370000000000000000000FFFF00FFFF00AA5572
:101380000000000000000000FFFF00FF3F409AB592
:10139000AAB4A8B0A8B0A8B0A993403F0D0D0D0DF8
:1013A0000D0D0D0D0D0D0D1DFDF902FCA830A04019
:1013B0000000000000000000FFFF00FF0D06030119
:1013C0000000000000000000FFFF00FFA8B0A8B070
:1013D000A8B0A8B0A8B0A8B0A993403FFC02A94DFE
:1013E0000D0D0D0D0D0D0D0D0D0D0D0DFF00AA5563
:1013F000000000000000000040A05020FF00AA559F
:10140000000000000000000003070E0C3F409AB5EA
:10141000A8B0A8B0A8B0A8B0A8B0A8B0D0BAB3CDB2
:10142000ADB3B6C4BAB7D7C29CBEBEDC2A45EB95F5
:10143000AFD5EB976B5DEB95AF576B37EFE7EFE70A
:10144000EFC01ECEDECEDEC0CFC70FE778397839C9
:101450007839783B7903391B391B3801FF00550077
:1014600000DB00000000FF00FFFF00FFFF00550051
:1014700000B600000000FF00FFFF00FF2D2D2D2D06
:101480002D2D2D2D2D2D2D2D2D2D2D2DA484A084F4
:10149000A480A484A084A480A484A084050203035F
:1014A0000003030CDFDFDFDFFFFFFFFFFFFFDFDFF6
:1014B000DFDF0C307FFFFF7F3F1F1F1F1F3F7FFFBE
:1014C000FF7F3010100C9F5151517171717171710A
:1014D0005151519F0C304FB49549301510101530B3
:1014E00049B5944F30100800000D181070D8888846
:1014F000D870121A0D020200020D1A1070D88888D6
:10150000D870101A0D020002020D1A1270D88888C5
:10151000D87010180D0000EE023200BC023200EE4E
:10152000023200BC023200EE023200BC023200EE97
:1015300002320000801210C0380CC6F2FB1D0D07ED
:10154000030100000000000000030C1831674F4E3B
:10155000DCF8D8F05070706020202000000000807F
:10156000C0E0F0F8FCFEFFFF7F3F1FE3F7FF7F3F87
:101570007FFFFF0F070301000000001010000000B4
:10158000000080C0E0F0783C9E4F27130FC0E1734D
:101590003E13173B690402010000000000080881A7
:1015A000667E3C3C7E668112100000000000000058
:1015B0000103070D1DFBF2C60C38C020202060700F
:1015C0007050F0D8F8DC4E4F6731180C031F3F7F86
:1015D000FFFFFEFCF8F0E0C080000000000000000B
:1015E000000103070FFFFF7F3F7FFFF7E310100F9E
:1015F00013274F9E3C78F0E0C08000000000000000
:1016000000000000010204693B17133E73E1C07E35
:10161000FFFFBDBD7E3C3C3C3E3E3C3C3C7C7C10E8
:10162000083C6ECB99895A3C08182C1C08180838BD
:10163000387C7C3C3C3C3E3E3C3C3C7EBDBDFFFFA0
:101640007E100838380818081C2C18083C5A89994C
:10165000CB6E3C08030205020202020705080305DF
:10166000070202020205021F1F000080C040D0587E
:10167000DC5CDE5EDE40DF55DF5F1FDF5EDE5EDCF2
:101680005CD850C040800000F0FEFFFFFFFFFFFF6E
:10169000FFFFFFFFFFFFFFFFFFE0AFE5AFEFAFEFA3
:1016A000AFEFAFEFAFEEE0062AEEEAEEEAEEEAEEDB
:1016B000EAEEEAEEEAEEEAEEEA80BEAABEBABEBA08
:1016C000BEBABEBA3E060000000101050D151D356B
:1016D0003D357D757D757D757D353D351D150D055A
:1016E00001010000000F0F4070786A7B6B7B6B7B01
:1016F0006B7B6A7870402F6D2F0D2F6D2F0D2F6D26
:101700002F0D2F6D2F0202030303030707070404A5
:101710000F0F0F0F05051F1F1F1F1F464143494C89
:10172000495459005448452054455354494E4700A4
:101730004553434150450050524553532042205495
:101740004F2053484F4F540047554E20534B494C60
:101750004C005052455353204220544F2041545482
:1017600041434B0053574F524420534B494C4C007C
:10177000484954204120545749434500444F55425D
:101780004C45204A554D5020534B494C4C0050522B
:1017900045535320555020414E4420444F574E004E
:1017A0004C4F4F4B20534B494C4C000808FF81A530
:1017B0006666A581FF0808FF81A9AAAAA981FF087A
:1017C00008EF919991B9D5B9D70808FF81A15E7D3D
:1017D000A181FF594F552048415645204245454E6D
:1017E0002044455354524F5945440054494D4520D7
:1017F0005041535345443A004D454348414E4943B7
:101800005300594F552044454645415445442054C2
:1018100048450090011400C2011400DB011400C20D
:10182000011400008096001400C8001400FA00148F
:101830000000808A021400BC021400EE0214002092
:1018400003140052031400840314000080C8001E17
:1018500000FA001E000080F4010A0058020A00BCD1
:10186000020A0020030A0084030A0020030A00BCC5
:10187000020A00E80332000080070DF00004F801BE
:1018800002FC01000403100807200D40E0F00000F6
:10189000000000F8F8F8F8F8F8FCFEFF000000007F
:1018A0000000000000000000F0E040000001000027
:1018B000000000030303030303070F1F00000000E1
:1018C000000000000000000001000031140C8E9F99
:1018D0003F37A7E7ECCC0086FE202036FEF004FE62
:1018E000E72321F3B21C00F88E020383C7FE00FE3B
:1018F000030306C6FC003FFE0C18301CBEFF0203AB
:101900000301B1F94161301803E1B02060C300F078
:101910004303F0C000C3E330101133630191F08042
:101920008183C2F301101033F1E030301001030065
:101930000000000F070302060C000F030000010760
:101940000F03000E0F0003070C090B0B0F000F070E
:101950000001010F0F000000000F07000000000051
:10196000080B00020202000009040000010202004C
:1019700000052400100105240101010424020605CC
:10198000240600010705810310004009040100023C
:101990000A0000000705020240000007058302401C
:1019A00000000403090412010002EF020140412378
:1019B000368000010102030141726475696E6F2077
:1019C0004C4C430041726475696E6F204C656F6EBC
:1019D0006172646F00002E2111241FBECFEFDAE088
:1019E000DEBFCDBF11E0A0E0B1E0EEEDFDE602C04C
:1019F00005900D92A837B107D9F729E0A8E7B1E023
:101A000001C01D92A936B207E1F71CE0CCEEDCE084
:101A100004C02197FE010E94D336CB3ED107C9F7FF
:101A20000E945B210C94ED360C9400008091E4043C
:101A300008956F927F928F929F92AF92BF92CF92B2
:101A4000DF92EF92FF920F931F93CF93DF936C017E
:101A5000CB013A017E2DFA01649131965491F2E066
:101A60006F0E711CC62FD0E0222301F1E1E0F0E0FF
:101A7000352F377011F4F0E0E0E0A52FA695A6957C
:101A8000A695AE0FBF2FB11DAC9FF001AD9FF00D1D
:101A9000BC9FF00D1124733011F4EE0FFF1F2E9F29
:101AA000D0012F9FB00D11246A0E7B1ED601AC0F02
:101AB000BD1F1A161B060CF069C020E8C216D1041F
:101AC0000CF064C09C01250F311D121613060CF09A
:101AD0005DC0803491050CF059C06114710409F4A3
:101AE00055C0382F3770FC0197FD379623E0F595E8
:101AF000E7952A95E1F72E2F97FF04C0332311F0C5
:101B00002FEF2E0FEE27FF27EC19FD09D7FC02C09F
:101B1000F0E0E0E090E89C19A038B1050CF4962FB5
:101B20009E1BA22F022E000CBB0B4A2F40952F3F6D
:101B30000CF040E0BB24B394852F877009F4B12CDE
:101B4000569556955695B50EAB0DB11D19971CF0CF
:101B500058E0B52EB21AB41A240F50E82503D0016C
:101B60001124AC0DBD1DAE0FBF1F649FE00DF11D14
:101B700011246E0E7F1EC32E032E000CDD08723062
:101B800009F448C090F4713009F48DC0DF91CF9111
:101B90001F910F91FF90EF90DF90CF90BF90AF908B
:101BA0009F908F907F906F900895733009F4C4C018
:101BB0000B2D020F7A3F51F7021741F3BD016B5F06
:101BC0007A4FF12CE12CE91608F067C0F301EE0D15
:101BD000FF1DE491F0E0AF010C2C02C0440F551F33
:101BE0000A94E2F727FD04C0FB018081842B8083E7
:101BF000332351F0273044F45B01F0E8AF0EB11C01
:101C0000F5018081852B8083FFEFEF1AFF0A6F5F5C
:101C10007F4FD9CF6FEF70E0032E02C0660F771FA2
:101C20000A94E2F760957095972E8B2C820E2815FA
:101C300009F4ACCF8D010B5F1A4FF12CE12CE916A2
:101C400030F5F301EE0DFF1DE491F0E0AF010C2C37
:101C500002C0440F551F0A94E2F727FD05C0F801A2
:101C600080818623842B8083332359F027304CF4E2
:101C70005801F0E8AF0EB11CF50180818921852B58
:101C80008083FFEFEF1AFF0A0F5F1F4FD8CF2F5F40
:101C90006C0E7D1EA058BF4FCACF2F5F6C0E7D1EED
:101CA000A058BF4F89CF0E0F1F1F8B2D820F821799
:101CB00009F46CCFBD016B5F7A4FF12CE12CE91672
:101CC00098F5F801EE0DFF1DA490B12C0C2C02C06C
:101CD000AA0CBB1C0A94E2F7A094B094F301EE0D99
:101CE000FF1D8490912C0C2C02C0880C991C0A9426
:101CF000E2F727FD08C0FB014081E42FEA214E2FC7
:101D00004829FB014083332349F027303CF4FB0191
:101D1000E058FF4FA080BA20B928B082FFEFEF1A39
:101D2000FF0A6F5F7F4FCBCF2F5F6C0E7D1E0C0FB6
:101D30001D1FA058BF4FBBCFE92EF12CE60DF71D9C
:101D4000AB5FBA4F60E870E06E197F09CE19DF090A
:101D5000AE01440F551FC1E0D0E07E01032E01C04B
:101D6000EE0C0A94EAF7192F0B2D892E932ECF93A0
:101D7000DF93ED01EF96EF962296A590C5909920FE
:101D800059F0AE9C5001CE9C600127302CF4F880B5
:101D9000D094FD20FB28F99222233AF0FC90C094C5
:101DA000FC20FA28FD920C94D60E11961A9529F76C
:101DB0000A9551F0182D23951124E40FF11DA60F5B
:101DC000B11DC60FD11DD9CFDF91CF911124DECE29
:101DD000E5E0F5E0A0E0B8E000800EBC8111012C48
:101DE0001197A0FDFDCF0192B9F70DB408959C01A4
:101DF000CB018770992791E001C0990F8A95EAF786
:101E000077FF02C0695F7F4FFB0183E0F595E7959F
:101E10008A95E1F7F695FE2FEE27F795E795E20F05
:101E2000F31FEB5FFA4F415030F08191DF011197C2
:101E3000892B8C93F8CF0895FC01809104058823A9
:101E400011F13FB7F89482E08093E9002091F2000D
:101E5000822F90E01816190614F481E090E0882390
:101E600039F0289844E6409303054091F1004083FF
:101E7000222339F02091F200211103C02BE6209398
:101E8000E8003FBF08958FEF9FEF08952FB7F894B4
:101E900083E08093E9009091E800892F807295FF9C
:101EA00004C09091F20080E4891B2FBF08958091B7
:101EB000FB0481110DC082E08093F70484E08093DD
:101EC000F8041092FA041092F90481E08093FB0464
:101ED00087EF94E00895CF93DF931F92CDB7DEB7DD
:101EE0006983DC01ED91FC910280F381E02D41E0FA
:101EF00050E0BE016F5F7F4F09950F90DF91CF914A
:101F0000089583E08093E9008091F200882319F01E
:101F10008AE38093E80008950E94460F90E00895B8
:101F2000CF93DF931F92CDB7DEB7FC0184859585F3
:101F300097FD08C02FEF3FEF358724870F90DF9183
:101F4000CF910895CE0101960E941C0F019719F4BC
:101F5000898190E0F3CF8FEF9FEFF0CF0F931F9326
:101F6000CF93DF931F92CDB7DEB78C01FC01848540
:101F7000958597FF0BC0CE0101960E941C0F01971B
:101F800071F4898190E0F80195878487F801848550
:101F900095850F90DF91CF911F910F9108958FEF4D
:101FA0009FEFF1CFFC018485958597FD0BC09FB70E
:101FB000F89482E08093E9008091F2009FBF90E066
:101FC000019608959FB7F89482E08093E90080918C
:101FD000F2009FBF90E008954091F1045091F20407
:101FE0002091EF043091F00442175307B4F490911C
:101FF000E8009570E1F39091E80092FD19C080939C
:10200000F1008091F1049091F20401968F73992769
:10201000892B19F48EEF8093E8008091F104909160
:10202000F20401969093F2048093F10481E0089504
:1020300080E00895DF92EF92FF920F931F93CF936A
:10204000DF93D82E8A01EB017B01E40EF51ECE153D
:10205000DF0559F0D7FE12C0FE0184910E94EC0FFB
:1020600021968111F4CF0FEF1FEFC801DF91CF91BF
:102070001F910F91FF90EF90DF9008958881EECF30
:102080000F931F93CF93DF931F92CDB7DEB782E0FC
:10209000898342E450E060E679E180E80E941A100A
:1020A0000E94570FDC0112960D911C91011511052C
:1020B00089F0D801ED91FC910280F381E02DBE0101
:1020C0006F5F7F4FC801099597FD04C0F801008537
:1020D0001185ECCF89810F90DF91CF911F910F91E6
:1020E0000895615030F02091F100FC0120830196A9
:1020F000F8CF289884E68093030508953FB7F894B5
:102100008091EB049091EC04A091ED04B091EE0469
:1021100026B5A89B05C02F3F19F00196A11DB11D42
:102120003FBFBA2FA92F982F8827BC01CD01620F7E
:10213000711D811D911D42E0660F771F881F991F39
:102140004A95D1F708958F929F92AF92BF92CF9206
:10215000DF92EF92FF926B017C010E947E104B0197
:102160005C01C114D104E104F104B9F00E947E10B5
:10217000681979098A099B09683E734081059105B0
:1021800080F321E0C21AD108E108F10888EE880E38
:1021900083E0981EA11CB11CE4CFFF90EF90DF906C
:1021A000CF90BF90AF909F908F9008958F929F9205
:1021B000AF92BF92CF92DF92EF92FF920F931F9355
:1021C000CF93DF936C017B018A0180911C018823EE
:1021D00009F45CC080910405882309F457C08091FC
:1021E000F60480FF05C08091E00082608093E000EB
:1021F000E801B12C8AEFA82E93E0892E2AE3922ED3
:10220000209711F4BB20D9F10E94460F81110AC01A
:10221000AA94AA20D9F161E070E080E090E00E94E9
:10222000A310EECF8C171D0611F00CF08C2F9FB76A
:10223000F8948092E9002091E80025FD02C09FBF3C
:10224000DFCF282F30E0C21BD30BF701815020F0E5
:1022500041914093F100FACFE20EF31EBB2021F032
:102260009092E800B12CEBCF8091E80085FDE7CF9C
:102270009092E800BB24B394209709F3F3CF5D98C4
:1022800084E68093F504101611063CF081E090E09E
:10229000F6019383828310E000E0C801DF91CF91C3
:1022A0001F910F91FF90EF90DF90CF90BF90AF9074
:1022B0009F908F900895AF92BF92CF92DF92EF924E
:1022C000FF920F931F93CF93DF936C017B018B01E0
:1022D000040F151FEB015E01AE18BF08C017D10730
:1022E00059F06991D601ED91FC910190F081E02DBA
:1022F000C6010995892B79F7C501DF91CF911F910F
:102300000F91FF90EF90DF90CF90BF90AF90089526
:102310006F927F928F929F92AF92BF92CF92DF92F5
:10232000EF92FF920F931F93CF93DF934C017B01AA
:10233000C22F102F98E0A92EB12C642E66946694BB
:102340006694712CCA0187709927892B79F5D4017D
:1023500017962D913C91C7019927B9010E94BF366C
:10236000269DF001279DF00D369DF00D11248E0F56
:102370009F1FD4011596ED91FC91E80FF91F208164
:10238000111112C0C095C223C083DF91CF911F915C
:102390000F91FF90EF90DF90CF90BF90AF909F9004
:1023A0008F907F906F900895C22BEECFD0E0477052
:1023B000C42ED12C83E0660C771C8A95E1F79E0130
:1023C00001C0220F4A95EAF7012FA301B701C4010A
:1023D0000E948811A301485F5F4FC5018C199D09B8
:1023E00002C0D595C7958A95E2F7A7CF5F926F9205
:1023F0007F928F929F92AF92BF92CF92DF92EF9295
:10240000FF920F931F93CF93DF93EC016A30F1F4A7
:102410008D859E859C878B878C892F853889820F37
:10242000932F911D988B8F8781E090E0DF91CF9162
:102430001F910F91FF90EF90DF90CF90BF90AF90E2
:102440009F908F907F906F905F900895AB84BC8435
:10245000693031F429E0A20EB11CBC86AB86E4CF12
:102460003DEFA3163FEFB3060CF45DC08F81988556
:10247000A816B9060CF057C0CF84D8888DEFC816BF
:102480008FEFD8060CF44FC089859A85C816D906F7
:102490000CF049C0603208F46FE780EE860F9FE9C8
:1024A000960F9A3118F49FEFC91AD90A8C3011F09F
:1024B0008B3119F42FEFC21AD20A869534E0839F2C
:1024C000C00111249C012C53304F7901912C812C97
:1024D000162F1170F701E80DF91D549011112DC040
:1024E000352D3F70532E3501680C791C8C81882363
:1024F00061F001E089899A89892B09F000E02FE0D9
:10250000A601B301CE010E9488110989252DA601DB
:10251000B301CE010E9488118FEF881A980A94E0C7
:1025200089169104B9F68B8990E004962B853C8539
:10253000820F931F9C878B8777CF52948FE058220E
:10254000D2CFEF92FF920F931F93CF93DF938C0123
:102550007B01D0E0C0E0F701EC0FFD1F6491662322
:1025600039F0C8010E94F611892B11F02196F3CFA2
:10257000CE01DF91CF911F910F91FF90EF900895C1
:1025800020918C01E0918A01F0918B01CF0102969C
:1025900090938B0180938A01222319F08591949165
:1025A0000895808191810895CF92DF92EF92FF92FA
:1025B000CF93DF930E94C012811520E8920791F417
:1025C000809171008D7F80937100109291004698E8
:1025D000479810928901DF91CF91FF90EF90DF90A3
:1025E000CF90089521E020938901813020E892075F
:1025F00051F4809187019091880190938B01809391
:102600008A010E94C01297FD05C0209186012223F5
:1026100009F454C020918501211150C021E020937C
:102620008D01EC01DF77209709F04BC081E08093AA
:102630008E0146983FE9C32E3FE0D32EE12CF12CCA
:10264000CAEFD0E0E0916309F09164090995811126
:1026500003C081E080938E0180918D01882329F051
:1026600080918E01882309F43FC047980E94C012D0
:102670000097F1F19C01DE010E94B036DC01CB0134
:1026800029E0B595A795979587952A95D1F710924A
:1026900090002AE020939100D0929900C092980077
:1026A00080938F0190939001A0939101B093920138
:1026B000809171008260809371008DCF10928D01A6
:1026C000B0CF9E0150E040E060E472E48FE090E023
:1026D0000E945C3669017A0181E0C81AD108E108DC
:1026E000F10810928E01AECF4699BFCF479ABECF68
:1026F0008FEF9FEFDC01CBCF9C01E1E7F0E0908111
:102700009D7F908381E080938C0130938B01209397
:102710008A0130938801209387010C94D412EF92A0
:102720000F931F933AEFE32E10E000E00E94190D83
:102730001F910F91EF900895EF920F931F9332E046
:10274000E32E10E000E00E94190D1F910F91EF9011
:1027500008952D9A0895BC0190E080E00C94A31098
:102760008FB18095807F669B88601C9B84600895F4
:102770001092E4043E983F9808953E9A3F9A81E073
:102780008093E404089580E0E5E0F5E081118FEFA7
:10279000002481938193819381930394D1F71092C4
:1027A0008401109283011092820110928101089598
:1027B000EF92FF920F931F93CF93DF93CDB7DEB7C6
:1027C0002C970FB6F894DEBF0FBECDBF49835A8356
:1027D0006B837C839E83EF82F88609871A872B8719
:1027E0003C8729813A814F815885820F932F911D13
:1027F00048175907D4F48B85840F952F911D2817FE
:1028000039079CF44B815C8169857A858E81840FC0
:10281000952F911D6817790744F42C85260F372FC3
:10282000311D81E0421753070CF080E02C960FB663
:10283000F894DEBF0FBECDBFDF91CF911F910F91F6
:10284000FF90EF900895CF93C82F0E94B013C82334
:1028500081E009F080E0CF910895CF93C82F0E94C6
:10286000B013982F9C2381E09C1380E0CF910895B2
:1028700080E00C94E80E80389105B8F4603471055E
:10288000A0F420E191E061FD94E060FD990F62FD0C
:102890009295687F269FD0011124A80FAB5FBA4F95
:1028A0008C9140FF03C0892B8C93089590958923C8
:1028B000FBCFEF92FF920F931F93CF93DF938C0187
:1028C000C62F462F61E070E00E94F70E4C2F68E0A3
:1028D00070E0C8010E94F70EEE24E394F12C41E071
:1028E000B701C8010E943B148FEFE81AF80A89E08B
:1028F000E816F104A1F7C00FD12FD11D219701E0F7
:1029000010E041E0B801CE010E943B140F5F1F4F61
:1029100009301105B1F7DF91CF911F910F91FF9011
:10292000EF9008958F929F92AF92BF92CF92DF92D5
:10293000EF92FF920F931F93CF93DF936D3089F047
:10294000C0908301D09084016A30D1F4109282014A
:102950001092810188E0C80ED11CD0928401C092EF
:10296000830181E090E0DF91CF911F910F91FF9063
:10297000EF90DF90CF90BF90AF909F908F90089591
:102980000091810110918201E5E06E9FE001112428
:10299000CC53D54F4801F12CF5E0E12CFF1629F07E
:1029A000CE010196FE01E490EC01B12CA12C4E2D3C
:1029B0004170B6016A0D7B1DC4010E943B14E69470
:1029C000FFEFAF1ABF0A88E0A816B10481F7F394AD
:1029D000EFEF8E1A9E0AF6E0FF12DECF0A5F1F4F5E
:1029E0001093820100938101BCCF81E0809310019C
:1029F0001092800110927F0124E030E030930301B7
:102A00002093020122E030E0309301012093000185
:102A100028EB31E030937E0120937D0120E832E005
:102A200030930D0120930C0126E331E030930B012C
:102A300020930A0193E090930501109203021092F3
:102A400002021092F9011092F80180930E01109287
:102A5000E1011092E0011092E2011092E501109262
:102A600027021092E0041092E50408958091F60187
:102A70009091F701805892409093F2018093F10178
:102A80008091F4019091F501805491409093EE0172
:102A90008093ED01809102019091030140EA489FEB
:102AA0009001499F300D1124205531093093AE0417
:102AB0002093AD046091000170910101469FC00117
:102AC000479F900D1124805591099093AC048093F9
:102AD000AB0440917D0150917E01240F351F30934E
:102AE0000302209302029093F9018093F8018091F0
:102AF0007C01883131F420E830E030930B022093E0
:102B00000A0290917B01983139F520EA30E0309348
:102B10000902209308028C3019F520E230E030934E
:102B20000B0220930A029C3071F420E430E03093D1
:102B3000090220930802863071F420EF3FEF3093B2
:102B40000B0220930A02963031F480E190E09093DA
:102B500009028093080208958C30F9F29C3029F321
:102B6000863089F7EACF8EEA9AE00E947C138AEFDA
:102B70008093E10481E08093C90484E68093DD04BE
:102B80008CE99FEF909346028093450290934A020E
:102B9000809349020895E0919701F0919801EE0F1A
:102BA000FF1FDF01A95EBD4F8D919C911197209170
:102BB000AD043091AE04281739071CF4C0968D93EC
:102BC0009C93E95EFD4F80819181821793071CF4ED
:102BD000C0979183808308952091AD043091AE0415
:102BE0008091A4049091A504821793072CF48097F8
:102BF0009093A5048093A4048091A4049091A504CB
:102C0000281739072CF480969093A5048093A40488
:102C10000895CF93DF9380917C0120917A014091B8
:102C20007B01E42FE150FF0BBF01A2E6B2E0FD0102
:102C300090E0891311C030917901F8E18F9FC001B4
:102C4000112420E04997421779F03D93FD01E80FE8
:102C5000F91F30832F5FF7CF2083EF01C60FD71FF7
:102C600028839F5F7896E5CFDF91CF9108952F92CB
:102C70003F924F925F926F927F928F929F92AF920C
:102C8000BF92CF92DF92EF92FF920F931F93CF9359
:102C9000DF93CDB7DEB76A970FB6F894DEBF0FBEED
:102CA000CDBF22E632E088E1F90110E010821F5F1B
:102CB00078961831D9F781502F5F3F4F8111F4CFAB
:102CC00010922002109221021092220210925F02B2
:102CD00010926002109261021092DF041092DE04E2
:102CE0001092C4011092BF011092BA011092B50166
:102CF000E0907C01EB8280EAE89E90011124309301
:102D00000D0220930C02F0907B01F982F89EC00125
:102D100011249093FB018093FA0135952795309308
:102D2000F7012093F601959587959093F50180938F
:102D3000F4010E94361586E180937A0187E1809341
:102D400079010E9409168EE1809362022981215047
:102D5000330BC901F901EE59FD4F2FE120834B815F
:102D60004150550B149FF001159FF00D1124EE59A1
:102D7000FD4F2CE12083E80FF91F8DE18083E09067
:102D80001001E9828E2D8450823018F00E2D08300B
:102D900039F480E280937A01809379010E940916C8
:102DA00019811B3031F410927A01109279010E943E
:102DB000091640917F015091800109810150110B4A
:102DC000F801EE0FFF1FEF5CFE4F80819181840FB1
:102DD000951FFC0164914F5F5F4FF3E06F9FB0015F
:102DE000112430E020E0DC01139626173707B1F0FC
:102DF000FC013196E4900296FC018491FD019491CE
:102E000018E1F12EFE9CF0011124EE59FD4FE80F60
:102E1000F11D90832D5F3F4FCD01E5CF240F351F6E
:102E20003093800120937F018090A4049090A504AA
:102E30000091A2040A871091A3041B872091A60485
:102E40002887309127023D8B4091B601488B5091E5
:102E5000B701598B8091B8018E879091B9019F87F6
:102E6000A091E501AC8BA090BB01B090BC01B091EA
:102E7000BD01BA8B7090BE01E091E201EB8B5090E6
:102E8000C0014090C101C090C201D090C301F09137
:102E9000E004FE8B3090B1012090B201E090B301CC
:102EA000EC86F090B401FD8619861D821C821E827C
:102EB0001F821B82F0E0E0E070E060E030E020E0A4
:102EC00040EA429F8001439F100D1124188F0F8B01
:102ED0008901B4E0000F111FBA95E1F7C9018E59BD
:102EE0009D4F9A8F898F90E080E0A98DBA8D6C906C
:102EF000B3E06B128FC0AB01405E5D4FDA016C92A4
:102F0000AB01440F551FDA01A95EBD4FBA83A983F7
:102F1000BAE0B89F7001B99FF00C1124A981BA8161
:102F2000ED92FC924F5E5D4FEF88F88CDA01ED92E6
:102F3000FC926F5F7F4FA98DBA8D5896BA8FA98F7B
:102F400040968038B1E09B0781F62F5F3F4F2831D4
:102F5000310509F0B5CFEB81E093C4015092C00177
:102F60004092C101C092C201D092C301FF81F0938F
:102F7000B5013092B1012092B201EC84E092B3012C
:102F8000FD84F092B4010E810093BA011889109368
:102F9000B60129892093B7013E853093B8014F854A
:102FA0004093B9018C819D819093DF048093DE046E
:102FB0009092A5048092A4049A859093A204AB8574
:102FC000A093A304B885B093A604E985E093BF015C
:102FD000A092BB01B092BC01FA89F093BD0170923E
:102FE000BE016A960FB6F894DEBF0FBECDBFDF916B
:102FF000CF911F910F91FF90EF90DF90CF90BF90F6
:10300000AF909F908F907F906F905F904F903F9088
:103010002F900895BAE0FB2E6F101DC0AF01415AEA
:103020005D4FEE24E394DA01EC92AF01440F551F9B
:10303000DA01A75ABD4F689E7001699EF00C1124F9
:10304000ED92FC924D5A5D4FEF88F88CDA01ED92CB
:10305000FC92319670CF5BE0F52E6F1011C04AE004
:10306000489F4001499F900C11245F895A87A88D81
:10307000AB87B1E0B88742E350E05D834C835BCF20
:1030800054E0651209C0AB89A11155CF582E492EC5
:103090006801B1E0BB834FCF45E0E42E6E1009C05C
:1030A000FC88F11048CF5C010A8B712E41E0498702
:1030B00042CF56E065120AC0AD89A1113CCF888B82
:1030C000998B0E871F87B1E0BE8335CFEE24E39442
:1030D0006E1031CFFE88F1102ECF382E292E0C879E
:1030E0001D8741E04F8327CF282F2150330BF90153
:1030F000EE0FFF1FEF5CFE4F8081918120917F01D9
:1031000030918001FC01E20FF31FE491E0937C0118
:10311000F9013196E80FF91FE491E0937B012E5FEE
:103120003F4F3093800120937F01089510928001DA
:1031300010927F0110927E0110927D011092780111
:103140008EE18093DD0180911001813009F580913D
:10315000AD049091AE04883E23E092070CF079C153
:103160008BE090E0909303018093020182E090E075
:10317000909301018093000188E99EEF90937E0176
:1031800080937D0183E08093100181E0809378013A
:1031900080911001823009F08FC1809178018111F6
:1031A0008BC18091AD049091AE049C01215D3740AC
:1031B0002532324008F065C183E090E0909303012E
:1031C0008093020181E090E09093010180930001DF
:1031D00010927E0110927D0186E08093100181E0C3
:1031E0008093780180911001843029F580917801D5
:1031F000811141C08091AB049091AC04893E23E0E1
:1032000092070CF49AC185E190E0909303018093BA
:10321000020181E090E0909301018093000182E03F
:10322000809310018CE99FEF90937E0180937D0144
:1032300081E080937801809110018530E1F48091E4
:103240007801811118C08BE090E090930301809386
:10325000020183E090E0909301018093000184E0FB
:103260008093100188E99EEF90937E0180937D0109
:1032700081E080937801809110018630F9F480918B
:10328000AB049091AC04843F41E094070CF074C10E
:103290008EE090E0909303018093020184E090E03F
:1032A000909301018093000182E0809310011092BD
:1032B0007E0110927D0181E0809378018091100160
:1032C000873029F580917801811121C08091AD046A
:1032D0009091AE04843F41E094070CF067C186E111
:1032E00090E0909303018093020184E090E090933A
:1032F00001018093000184E39EEF90937E0180930F
:103300007D0189E08093100181E0809378018091B4
:103310001001883029F580917801811121C08091B8
:10332000AD049091AE04883542E094070CF054C18E
:1033300084E190E0909303018093020186E190E0A4
:10334000909301018093000180EC9EEF90937E01A9
:1033500080937D018BE08093100181E08093780160
:1033600080911001893029F580917801811121C067
:103370008091AD049091AE04883542E094070CF042
:1033800043C183E090E0909303018093020186E1C2
:1033900090E0909301018093000188E092E0909387
:1033A0007E0180937D018AE08093100181E080930B
:1033B0007801809110018A3019F58091780181118E
:1033C0001FC08091AD049091AE04883542E094070F
:1033D0000CF032C182E090E09093030180930201EF
:1033E000909301018093000184E690E090937E0128
:1033F00080937D0189E08093100181E080937801C2
:10340000809110018B30D1F480917801811116C028
:1034100082E090E090930301809302019093010178
:103420008093000180E491E090937E0180937D0180
:1034300088E08093100181E0809378018091F3010E
:1034400081111092F301809110010E9474180C9464
:103450003716883E934009F498CE81E090E090932F
:1034600003018093020184E090E090930101809336
:10347000000188E092E090937E0180937D0182E0DC
:1034800082CE843691050CF005C18BE090E09093DC
:1034900003018093020182E090E090930101809308
:1034A000000188E99EEF90937E0180937D0181E089
:1034B000809310018093780180911001833009F08E
:1034C00091CE809178018111B6CE8091AD0490911A
:1034D000AE04883E23E09207B4F485E190E0909337
:1034E00003018093020186E190E0909301018093B3
:1034F00000018AE08093100188E99EEF90937E019D
:1035000080937D016CCE883E934009F494CE81E097
:1035100090E090930301809302018AE090E0909301
:1035200001018093000181E08093100128E032E0E6
:1035300030937E0120937D0153CE883E934009F461
:103540009ACE8091AD049091AE04843F21E0920721
:103550000CF08AC088E090E0909303018093020110
:1035600084E090E0909301018093000188E08093D3
:10357000100188E99EEF58CE893E93400CF49ECE10
:1035800085E190E0909303018093020182E090E056
:10359000909301018093000187E08093100188ECF3
:1035A00090E090937E0180937D0185CE89329A4090
:1035B0000CF4ADCE82E090E0909303018093020181
:1035C00084E190E0909301018093000110927E01CC
:1035D00010927D0186E096CE8835924009F4C0CEE7
:1035E00082E090E0909303018093020181E090E0FB
:1035F000909301018093000188E092E090937E0116
:1036000080937D0184E0A7CE893E93400CF4D1CE17
:1036100081E090E0909303018093020183E090E0C9
:10362000909301018093000188E092E090937E01E5
:1036300080937D0187E0B8CE893E93400CF4E0CEC4
:1036400085E090E0909303018093020182E090E096
:10365000909301018093000180EC9EEF90937E0196
:1036600080937D0183E0C7CE893E93400CF4E3CD87
:1036700081E090E090930301809302018AE090E062
:10368000909301018093000185E08093100188E010
:1036900092E0CACD89329A400CF4A4CD84E090E047
:1036A00090930301809302018AE090E090930101DE
:1036B0008093000188E092E090937E0180937D01E9
:1036C00084E08093100181E0F5CE089590E080E0E1
:1036D00008958F929F92AF92BF92EF92FF920F93B5
:1036E0001F93CF93DF93CDB7DEB7A1970FB6F894B2
:1036F000DEBF0FBECDBF7C01FA01CB0119A2223083
:1037000008F42AE08E010F5D1F4F822E912CB12C00
:10371000A12CBF01A50194010E948E36F901CA01B6
:103720006A304CF5605DD8016E938D01232B242BFC
:10373000252B79F790E080E0109761F0FD01019072
:103740000020E9F73197AF014A1B5B0BBD01C701B0
:103750000E945B11A1960FB6F894DEBF0FBECDBFDD
:10376000DF91CF911F910F91FF90EF90BF90AF909D
:103770009F908F900895695CD6CFCF92DF92EF92A1
:10378000FF920F931F93CF93DF936B01770FEE0898
:10379000FF08F7FE1BC0EC016DE20E94F6118C01E0
:1037A00044275527BA014C195D096E097F092AE0A3
:1037B000CE010E94691B800F911FDF91CF911F9155
:1037C0000F91FF90EF90DF90CF9008952AE0B7011E
:1037D000A601DF91CF911F910F91FF90EF90DF90A5
:1037E000CF900C94691B0C9446362F923F925F92B7
:1037F0006F927F928F929F92AF92BF92CF92DF9201
:10380000EF92FF920F931F93CF93DF9381EC8093FE
:103810007C0085B1806F85B984B1877E84B984B11D
:10382000876E84B95E9A5F988AB1806D8AB9769AFC
:103830006E9881B3806F81BB899880B38D7080BB97
:1038400080E58CBD81E08DBD85E090E00E94AB13EA
:103850005F9A85E090E00E94AB135E985C98E1EA85
:10386000FAE084918EBD00000DB407FEFDCF3196C5
:103870004AE0EE3AF407A9F75C9A81E88093640085
:10388000809165008160809365000E94381480E813
:103890000E942D148823A9F05C9885EA8EBD000053
:1038A0000DB407FEFDCF5C9A2E982F982D9880912D
:1038B000640080628093640081E083BF889513BEBA
:1038C000FCCF84E00E942D14882309F448C02D9871
:1038D00084E80E942D148823E1F00E94A91388EC4B
:1038E00090E00E94AB132F9882E090E00E94463651
:1038F0008F3F29F06FEF82E090E00E944E3684EF18
:1039000091E00E94AB132F9A84E80E942D1481113C
:10391000FBCF84E10E942D148823E1F00E94A913BB
:1039200088EC90E00E94AB132E9882E090E00E9419
:103930004636882329F060E082E090E00E944E360F
:1039400084EF91E00E94AB132E9A84E10E942D1423
:103950008111FBCF88EC90E00E94AB13B2CF0E94A4
:10396000A91382E090E00E94F31B8823C1F10E941A
:10397000BD1381E090E00E94F31B81FF12C0582F1D
:103980005470552E82FD2E98C1EFDFEF08E010E055
:1039900080E40E942D14882329F12E9A2F9A0E94E8
:1039A000A91382E390E00E94AB130E94B01381112F
:1039B000F8CF80E180930401DF91CF911F910F91A7
:1039C000FF90EF90DF90CF90BF90AF909F908F903F
:1039D0007F906F905F903F902F900C9438140E94CE
:1039E000B813C7CF552029F0C430D10511F42E9A51
:1039F0002F9881E00E94E80E9E01D7FF04C0222785
:103A000033272C1B3D0B27703327CE01D7FD07969C
:103A100053E0959587955A95E1F7D7FF05C0019733
:103A2000F801E21BF30B9F01BC017695762F662708
:103A3000779567956B5F7A4FB0E0A0E03801621A26
:103A4000730A8E3FFFEF9F0709F43BC07B0150E0F4
:103A500040E0FD01EF50F64F5F014B01F0E88F0EA3
:103A6000911C8F3F980779F0F501E40FF51FE49161
:103A7000F0E06F01022E01C0CC0C0A94EAF7F701C6
:103A8000D488CD28C48A2115310599F0F501E40FB9
:103A9000F51FE4916401C40ED51EF0E01F01062C51
:103AA00002C0359427940A94E2F7F601348823285B
:103AB000248A4F5F5F4FFFEFEF1AFF0A4835510529
:103AC00081F60196A85ABF4F60587F4FA03BB105C1
:103AD00009F0B7CF0E9438148FE090E00E94AB133A
:103AE0002196C931D10509F053CF552011F02F9AF5
:103AF0002D9880E991E00E94AB130E94A91381E008
:103B000090E00E94F31B80FF4CCF8AE090E00E947F
:103B1000F31B9FEF980F9E3F08F043CF22E330E066
:103B2000309382012093810128E330E030938401B7
:103B300020938301CBE0D0E0682F85E699E00E94D6
:103B40009214CE010E94F31B2196C131D105A1F739
:103B50000E94381488EE93E00E94AB1322CF1F928C
:103B60000F920FB60F9211248F939F938091E100D3
:103B70009091E100937F9093E10083FF0FC010923A
:103B8000E90091E09093EB001092EC0092E39093A7
:103B9000ED001092040598E09093F00082FF22C09F
:103BA00093E09093E9009091F200992319F09AE341
:103BB0009093E8009091F504992341F09091F504D9
:103BC00091509093F504911101C05D9A9091030575
:103BD000992341F090910305915090930305911121
:103BE00001C0289A84FF18C08091E2008E7E816017
:103BF0008093E2008091E1008F7E8093E1008091CC
:103C0000F6048E7E80618093F6049F918F910F90D1
:103C10000FBE0F901F90189580FFF7CF8091E200A4
:103C20008E7E80618093E2008091E1008E7E8093A1
:103C3000E1008091F6048E7E8160E5CF1F920F92A5
:103C40000FB60F921124CF92DF92EF92FF920F9353
:103C50001F932F933F934F935F936F937F938F9314
:103C60009F93AF93BF93EF93FF93CF93DF93CDB722
:103C7000DEB76C97DEBFCDBF1092E9008091E800FF
:103C800083FF25C068E0CE0145960E94711082EF47
:103C90008093E8008D8987FF39C09091E80090FFFC
:103CA000FCCF982F907609F034C19E894F89588DAA
:103CB0002F89F88C911131C0803861F58091F4041E
:103CC0008093F1001092F1008EEF8093E8006C96E3
:103CD0000FB6F894DEBF0FBECDBFDF91CF91FF913D
:103CE000EF91BF91AF919F918F917F916F915F9174
:103CF0004F913F912F911F910F91FF90EF90DF9087
:103D0000CF900F900FBE0F901F9018959EEF90933D
:103D1000E800C7CF1092F100D5CF913059F481114E
:103D2000D3CF4130510581F68091F4048D7F80938B
:103D3000F404CACF933049F48111C6CF4130510504
:103D400019F68091F4048260F2CF953041F48091AD
:103D5000E80080FFFCCF20682093E300B5CF9630C9
:103D600009F0A9C00B8D1C8D22E01092E900109281
:103D7000F2041092F104F2122EC01092F00410928C
:103D8000EF040E9440101F8299E09983FA8291E02B
:103D90009E8390EA98879AEF99872091F104309159
:103DA000F204275F3F4F3C832B838D831092E90001
:103DB0001092F2041092F1041093F0040093EF04B7
:103DC00049E050E0BE016F5F7F4F80E00E941A1013
:103DD0000E94401079CF1093F0040093EF040E94EA
:103DE000570FDC0112960D911C910115110509F474
:103DF00051C1D801ED91FC910480F581E02DBE0107
:103E00006B5E7F4FC8010995009709F03EC1F8012C
:103E100000851185EACFF3E0FF120EC08F89882359
:103E200009F440C0823061F440E860E184EC99E13B
:103E30000E94FB20811148CF81E28093EB0047CFA5
:103E4000813029F440E86BE088EB99E1F1CF8330D1
:103E500099F70E94570FDC011296ED90FC908E01AD
:103E60000F5F1F4F6801E114F10479F0D701ED9164
:103E7000FC910680F781E02DB801C7010995080F74
:103E8000111DF701E084F184EECFD8011C92F601F8
:103E900001900020E9F73197BF016C197D0940E0DE
:103EA000C601C6CF62EA79E1FB01449150E080E8A7
:103EB0000E941A1009CF973009F4BECF983021F430
:103EC00081E08093F10000CF993009F0FDCE83703E
:103ED00009F0B2CFE4E5F1E081E031E096E3219131
:103EE000222371F08093E9003093EB00DF011197FA
:103EF0002C912093EC009093ED008F5F873079F741
:103F00008EE78093EA001092EA008F89809304057F
:103F1000DBCE8B8D9C8D1092E9001092F2041092F2
:103F2000F1049093F0048093EF04898D811192C085
:103F30008E899D89913A49F4813209F07DCF47E01D
:103F400050E065E171E080E0B3CF913209F074CFC9
:103F5000833269F48F89988DB0E0A0E080931101DD
:103F600090931201A0931301B0931401ADCE80324F
:103F700069F48091E80082FFFCCF67E085E191E081
:103F80000E9471108BEF8093E8009ECE823209F080
:103F90009BCE8F8980931C01EEEFFFE78591949172
:103FA0008B3F9C4D51F1E0E0F8E08091150190913C
:103FB0001601A0911701B0911801803B9440A10512
:103FC000B105F1F480911C0180FD1AC0EE3F8AE03A
:103FD000F80789F587E797E79183808380916000F0
:103FE0008093F30488E19BE00FB6F894A895809342
:103FF00060000FBE9093600067CEEEEFFAE0D5CF81
:10400000808191818737974709F05ECEA89580918E
:1040100060008861809360008091F3048093600069
:10402000EE3F2AE0F20789F08091FE0A9091FF0AA4
:104030009183808349CE808191818737980751F29F
:104040009093FF0A8093FE0AC5CF1092FF0A109248
:10405000FE0A3ACE0E94570FDC0112960D911C9178
:104060000115110509F4E8CED801ED91FC910190FC
:10407000F081E02DBE016B5E7F4FC8010995811173
:1040800023CEF80100851185EBCF181619060CF424
:104090001BCED2CEF1E0FF12BECE66EA79E104CFAC
:1040A0001F920F920FB60F9211242F933F938F936D
:1040B0009F93AF93BF938091E7049091E804A09100
:1040C000E904B091EA043091E60423E0230F2D3790
:1040D00058F50196A11DB11D2093E6048093E704D5
:1040E0009093E804A093E904B093EA048091EB0470
:1040F0009091EC04A091ED04B091EE040196A11D05
:10410000B11D8093EB049093EC04A093ED04B09365
:10411000EE04BF91AF919F918F913F912F910F909E
:104120000FBE0F901F90189526E8230F0296A11D31
:10413000B11DD2CF1F920F920FB60F9211242F9361
:104140003F934F935F936F937F938F939F93AF931F
:10415000BF93EF93FF9380918F0190919001A09175
:104160009101B0919201892B8A2B8B2B09F440C0CD
:1041700080918E0181110BC088B190E4892788B9A4
:1041800080918D01882319F088B1805888B9809179
:104190008F0190919001A0919101B0919201181618
:1041A00019061A061B069CF480918F0190919001CC
:1041B000A0919101B09192010197A109B109809359
:1041C0008F0190939001A0939101B0939201FF9180
:1041D000EF91BF91AF919F918F917F916F915F917F
:1041E0004F913F912F910F900FBE0F901F901895F8
:1041F0000E94D412ECCFEF92FF920F931F93CF93B4
:10420000DF93F82E192FE62E042F81E0860F880FFA
:104210000E94EC0F83E00E94EC0FCF2DD12FEC0E0B
:10422000FD2EF11CCE15DF05B9F007FF13C0FE010E
:1042300084910E94EC0F182F80E00E94EC0F8123E4
:1042400021968111EFCFDF91CF911F910F91FF90B8
:10425000EF9008958881EDCF81E0F5CFE5E0F9E0BA
:104260001382128288EE93E0A0E0B0E0848395830D
:10427000A683B7838EE591E0918380838FEF9FEFD4
:1042800095878487E5E6F9E01382128280E791E062
:104290009183808386E19DE0909364098093630914
:1042A00080E090E8909362098093610946983E9A75
:1042B00047983F9A0895CF93DF93CDB7DEB7E9973C
:1042C0000FB6F894DEBF0FBECDBF789484B5826080
:1042D00084BD84B5816084BD85B5826085BD85B5AA
:1042E000816085BD80916E00816080936E00109228
:1042F00081008091810082608093810080918100A3
:104300008160809381008091800081608093800033
:1043100080919100826080939100809191008160F2
:1043200080939100809190008160809390008091B3
:10433000C10084608093C1008091C100826080933D
:10434000C1008091C10081608093C1008091C30051
:1043500081608093C3008091C00082608093C00020
:104360008091C20081608093C20080917A00846055
:1043700080937A0080917A00826080937A008091A5
:104380007A00816080937A0080917A0080688093BF
:104390007A00109204051092F4041092F6048091B1
:1043A000D70081608093D70080EA8093D80089B5D8
:1043B000806189BD89B5826089BD09B400FEFDCFE9
:1043C00061E070E080E090E00E94A3108091D8004E
:1043D0008F7C80618093D8008091E000807F809303
:1043E000E0008091E1008E7E8093E1008DE080937B
:1043F000E200559A209A0E94F51B10EA412E512C9A
:104400008FB7F8944091E7045091E8046091E90473
:104410007091EA048FBF80919501882349F0109232
:10442000950180E090E0892B59F30E940000E8CFCD
:1044300080919601242E281A822D9091040129162C
:1044400040F48F5F891768F781E083BF889513BEBA
:10445000E8CF81E08093950140939601809193018C
:1044600090919401019690939401809393010E94FE
:10447000C3138091E504811142C020E04BEC58E168
:1044800060E170E080E290E00E949C1320E049E847
:1044900058E169E270E083E490E00E949C1380910F
:1044A000E404882349F020E049E758E169E270E03C
:1044B00086E590E00E949C130E94381480E40E94DC
:1044C0002D1481110E94BD1380E20E942D148111D0
:1044D0000E94B81388E00E942D14882309F4B9C300
:1044E000809110010E9474180E94371681E0809319
:1044F000E50484EF8093E30484E08093E2048091F8
:1045000009018F5F863009F4AAC380930901809165
:10451000E304882319F081508093E304809109011A
:10452000853089F48091E0019091E10101969093AA
:10453000E1018093E001809108018F5F843009F4EC
:1045400090C3809308018091E0019091E1016AE0BD
:1045500070E00E94BF367093DF016093DE018091AE
:1045600006018F5F843009F48AC38093060180912D
:10457000E104882309F44DC081508093E104813027
:1045800009F047C090910501915090930501911158
:104590003EC01C821B822BE431E03A83298325E054
:1045A00035E03F832E8320E830E03987288720E4F8
:1045B00030E03B872A8795E09D8B8C8B1F861E867B
:1045C000198A188A1D861C8681E090E09B8B8A8B55
:1045D0001D820E94C31385E090E09F878E879D8790
:1045E0008C878EE190E0998B888B63ED77E1CE012B
:1045F00001960E94A1120E94381488EB9BE00E9451
:10460000AB130E94C3130E9438140E94F5140E9439
:10461000361580912602882309F473C08150809357
:104620002602813009F06DC01C821B822BE431E030
:104630003A83298325E035E03F832E8320E830E06C
:104640003987288720E430E03B872A8795E09D8BD7
:104650008C8B1F861E86198A188A1D861C8681E00F
:1046600090E09B8B8A8B1D820E94C31304E110E0B3
:104670001F870E871D870C878AE090E0998B888BB7
:1046800062E078E1CE0101960E94A112B8E2CB2E41
:10469000D12CDF86CE86DD86CC86198B088B68EF21
:1046A00077E1CE0101960E94A1120EE110E01F8772
:1046B0000E871D870C87D98AC88A6BEE77E1CE01F9
:1046C00001960E94A1121F870E871D870C8722E387
:1046D00030E0398B288B6091E0017091E101CE01CF
:1046E00001960E94BD1B0E94381480E797E10E944A
:1046F000AB130E94C3130E943814109226020E942A
:10470000F5148091AF04882319F081508093AF0491
:104710008091DD01882319F081508093DD01809123
:10472000DD04882319F081508093DD048091DC043E
:10473000882319F081508093DC048091E104811179
:1047400031C381E08093EA012091AD043091AE0441
:10475000C90180569F4FB2010E94BF365B01E091B4
:10476000AB04F091AC04CF01CC96B2010E94BF36ED
:104770006B0188E18A9D80018B9D100D11240E59DB
:104780001D4FD801A60FB71F8C91853170F4CF0152
:10479000865A9F4FB2010E94BF36060F171FD801DD
:1047A0008C91853110F41092EA0181E08093E90147
:1047B000C901B2010E94BF3688E1869F8001879FB0
:1047C000100D11240E591D4FD801AC0DBD1D8C913B
:1047D000853170F4CF01865A9F4FB2010E94BF36D7
:1047E000060F171FD8018C91853110F41092E90142
:1047F00081E08093E401C9014E96B2010E94BF3668
:104800008B01CF010A96B2010E94BF366B0148E1CD
:10481000409FD001419FB00D1124AE59BD4FA60F4E
:10482000B71F8C918531A8F4C9018E579F4FB201F3
:104830000E94BF36469FC001479F900D11248E599C
:104840009D4FC80ED91ED6018C91853110F410925F
:10485000E40181E08093FF01CF0180569F4FB201B8
:104860000E94BF36FB0148E1409FD001419FB00D3F
:104870001124AE59BD4FA60FB71F8C918531A0F4FE
:10488000C9018E579F4FB2010E94BF36469FC0019B
:10489000479F900D11248E599D4FE80FF91F80817D
:1048A000853110F41092FF0180E40E942D148823BA
:1048B00021F180910E0110920F01811103C081E05E
:1048C00080930E0180910602909107028530910538
:1048D0002CF40196909307028093060280910602C1
:1048E000909107029C01255031092530310528F4AB
:1048F0000296909307028093060280E40E9423149C
:10490000882361F08091060290910702181619061B
:104910002CF40197909307028093060210910E01E8
:10492000112359F08091EA01882339F0109207028F
:104930001092060281E080930F0180E20E942D1404
:10494000882309F110920F01111110920E0180912C
:104950000602909107028C3FBFEF9B072CF0019756
:1049600090930702809306028091060290910702BD
:104970009C01275F3F4F2530310528F40297909323
:1049800007028093060280E20E942314882359F0D4
:10499000809106029091070297FF05C001969093BF
:1049A00007028093060280910E0181110BC0809155
:1049B000E901882339F0109207021092060281E083
:1049C00080930F0180E40E942314882341F080E249
:1049D0000E942314882319F081E080930F0188E05E
:1049E0000E942D148823E9F08091FE01811119C0E5
:1049F0008091FD018823A9F08091E801811111C007
:104A000081E08093E8018093FE011092FD011092F5
:104A1000FC018093E7011092E60183E398E10E9494
:104A20007C1388E00E942D14882309F18091E50110
:104A30008823E9F08091E801811119C08091E70194
:104A40008823A9F08091E601811111C081E0809353
:104A5000E8018093FE011092FD011092FC01809309
:104A6000E6011092E70183E398E10E947C1388E05D
:104A70000E942D149091E401882309F405C18091CE
:104A8000FE01882311F40C94D535911100C181E009
:104A90008093E8018091000290910102853EEFEF42
:104AA0009E070CF4EEC004979093010280930002DD
:104AB00088E00E942314882321F01092FE011092B6
:104AC000E80180912702882301F184E00E942D14DF
:104AD0008823A9F08091AF04811111C08091E30176
:104AE00081110DC08FE08093AF0483E198E10E94B3
:104AF0007C1385E08093DC0481E08093E30184E013
:104B00000E94231481111092E3018091E004882314
:104B100009F459C084E00E942D14882309F44DC083
:104B20008091E301811149C081E08093E301F0E4C9
:104B3000CF2EF2E0DF2E10E000E0A5E0BA2EFF2439
:104B4000F394D6018D916D01811132C08091AF0433
:104B500081112EC083E198E10E947C13B092DC04A5
:104B6000F6013197F082B3E0B093AF0480910E016B
:104B7000F801E25FFD4F882309F496C0F082C80176
:104B8000880F991FFC01E25DFD4F2091AD0430912B
:104B9000AE04205B3F4F31832083885D9D4F209181
:104BA000AB043091AC0422593F4FFC013183208388
:104BB0000F5F1F4F0330110521F684E00E9423147C
:104BC00081111092E3018091E201882351F100915B
:104BD000F8011091F90180E10E942D14882379F0E9
:104BE0008091FA019091FB018054914008171907B8
:104BF00034F4025E1F4F1093F9010093F80180E82E
:104C00000E942D14882369F08091F8019091F90198
:104C10008134F1E09F072CF04E979093F901809337
:104C2000F801809102029091030280589240E09135
:104C3000F101F091F201E817F907C4F58E1B9F0B03
:104C400069E170E00E94BF367093F0016093EF015C
:104C500030C084E00E942D14811142CCE2CB81E06F
:104C600054CC91E090930801809107018F5F8430CC
:104C700019F08093070167CC9093070164CC81E021
:104C800074CC1092FE0114CF992309F411CF8091B6
:104C9000FE0181110C94DB3510920102109200028A
:104CA00081E08093FC0104CF108269CF8E179F07AB
:104CB0002CF28091EF019091F001E80FF91F8091A3
:104CC000F8019091F901805491402091ED013091CB
:104CD000EE01281739075CF4821B930B6AE070E041
:104CE0000E94BF367093EC016093EB0103C0821702
:104CF000930794F38091EB019091EC01280F391FF9
:104D00008091DA049091DB048E0F9F1F9093F20143
:104D10008093F1014091D8045091D904240F351F9C
:104D20003093EE012093ED01EAE0F0E0BF010E9434
:104D3000BF3670934C0260934B02C901BF010E94C1
:104D4000BF3670934E0260934D028091AD049091F6
:104D5000AE04805B9F4FB2010E94BF369B018091E1
:104D6000AB049091AC04805B9F4FB2010E94BF36B0
:104D700088E1829FF001839FF00D1124EE59FD4FD1
:104D8000E60FF71F8081823019F491E09093F301D0
:104D90008750833010F40E94B3158091F301811184
:104DA0000E9496182091FD0121111AC04091AB0478
:104DB0005091AC048091FA019091FB01481759077A
:104DC0007CF481E08093FC018091000290910102CB
:104DD0008A3091052CF40296909301028093000290
:104DE0008091E10481110C94EF30409102025091C6
:104DF000030280914B0290914C0260910A027091E3
:104E00000B02861B970B9093440280934302809180
:104E10004D0290914E026091080270910902861B2A
:104E2000970B90934802809347028091AD04909134
:104E3000AE046091060270910702860F971F97FDDE
:104E400052C09093AE048093AD0480910C02909177
:104E50000D02FC01EF59F1096091AD047091AE04AF
:104E60006E177F075CF0BC01605A71097093AE0445
:104E70006093AD04109207021092060230910F0168
:104E800031110EC0E0910602F09107023BE13E9F16
:104E9000B0013F9F700D11247093050260930402CE
:104EA00030910E01332311F40C942030805892403D
:104EB0004817590714F00C942E304091AD045091CE
:104EC000AE04413832E0530714F40C942E30809134
:104ED000040290910502840F951F90930302809322
:104EE00002020C942E301092AE041092AD04109277
:104EF000070210920602A9CF1092AC041092AB04E4
:104F000010920102109200020C9440301092FD01A8
:104F100081E08093FC010C946B3080970C941431E9
:104F2000C9010A97B2010E94BF364B01469FC001DA
:104F3000479F900D11248E599D4F680E791ED30105
:104F40008C91853108F0F082C601B2010E94BF3613
:104F5000489DD001499DB00D1124AE59BD4FA60FFB
:104F6000B71F8C91853110F00C949731F0820C941E
:104F70009731255031090C949E31CF010A97B20127
:104F80000E94BF36F69EF001F79EF00D1124EE59F7
:104F9000FD4FE20FF31F8081853110F40C94F33143
:104FA000D501EC920C94F331029711F00C941E325F
:104FB000D801ED91FC91C901805B9F4FB2010E9425
:104FC000BF369B01CF01865A9F4FB2010E94BF3668
:104FD000F29ED001F39EB00D1124AE59BD4FA60F25
:104FE000B71F8C91853110F00C941E323A960C94B8
:104FF0001B3205970C942832C9010A97B2010E940E
:10500000BF3688E1869FF001879FF00D1124EE598D
:10501000FD4FE00FF11F8081853110F40C94673251
:1050200081E08093A6040C946732225031090C94DD
:105030006F321092DB041092DA041092D9041092AD
:10504000D8040C9468348130910551F4D6018D91C7
:105050009C9111972CA43DA4821993090C94E434DB
:105060008230910541F4D5018D919C9111972EA428
:105070003FA40C94E234039711F00C94E634D5016C
:105080008D919C91119728A839A8E6CF20E044EA99
:1050900050E10E949C13C801992011F40C94B7357B
:1050A00003968A199B0921E0F11003C020910801A1
:1050B000215044E850E10C9449352551B501681B55
:1050C000790B4AEB52E1C6018A1B9B0B0E949C1391
:1050D0005FEF651A750A60E1C60ED11C78E16716AC
:1050E000710411F00C94623580E1880E911C9FEFE1
:1050F000291A390AA6E88A16A1E09A0611F00C943A
:105100005535712C612CEEA1FFA18081882309F413
:1051100048C19301220F331FF901E95EFD4F8081E1
:1051200091816AE070E00E94BF366B01F901E1569F
:10513000FE4F71836083F901EF5EFD4F80819181A5
:105140006AE070E00E94BF365B0127563E4FD901EE
:105150006D937C9320904D0230904E023FAA2EAA70
:105160001B012EA93FA9221A330A80904B0290906E
:105170004C02A6014819590959A748A7EE24E394FF
:1051800003EA14E120E043EC54E1B10188A599A5BC
:105190000E94190DB5016E5F7F4F8EA99FA9681BF4
:1051A000790BF301E35EFD4F8081882309F485C606
:1051B000C601099620E04CE954E1881999090E943A
:1051C0008F138091E1048111ECC08091490290918C
:1051D0004A02E0914702F091480220914502309145
:1051E0004602A0914302B091440248A568A579A562
:1051F0007F8F6E8F622D39A228A270E17AA37BA3E4
:105200002A1B3B0BE22E3F8B2E8B8E1B9F0B082FF6
:10521000998F888F7A8F7B8FFF88198D20E130E1FD
:105220005F8D79A180E190E10E94D81381110E94E5
:10523000B3158091AF04882309F442C0209149023C
:1052400030914A028091470290914802281B390B05
:1052500080914502909146020A97409143025091F5
:105260004402841B950BE82E9A838983022F3C838A
:105270002B8384E28D8390E19E83FA801C8124E25B
:1052800030E14E8D5F8D68A179A18AA19BA10E941A
:10529000D8138823A9F087E598E10E947C13AEA17A
:1052A000BFA18C9181508C9370929801609297016C
:1052B0000E94CB15B1E0B093CA04E2E3E093DD04B1
:1052C0008091E004882309F46CC0B0E4AB2EB2E016
:1052D000BB2ED12CC12CD5018D915D01882309F401
:1052E00058C0F601E65CFD4F2081318180914D026E
:1052F00090914E02281B390BF601EC5CFD4F80812A
:10530000918140914B0250914C02841B950BE82EE9
:105310009A838983022F3C832B83B8E0BD83E3E02B
:10532000EE83FA801C8128E033E04E8D5F8D68A10A
:1053300079A18AA19BA10E94D813882351F187E506
:1053400098E10E947C13AEA1BFA18C9181508C93F7
:1053500070929801609297010E94CB15F5013197E8
:105360001082B1E0B093C804F601E25DFD4F808188
:1053700091819093AA048093A904F601E85DFD4F02
:10538000808191819093A8048093A704E2E3E09345
:10539000DD04F2E0CF0ED11C26E0C216D10409F0E4
:1053A0009ACF3FEF631A730A4EA15FA14F5F5F4F21
:1053B0005FA34EA353E06516710409F0A4CE712CCF
:1053C000612CA0E1BA2EAA24A394ACA1BDA18C911A
:1053D000882309F412C12090490230904A02E091DA
:1053E0004702F0914802FFA3EEA3809045029090FF
:1053F0004602E0904302F0904402F301E75AFD4F69
:10540000808191816AE070E00E94BF366B01F301F8
:10541000E555FE4F71836083F301ED5AFD4F8081A6
:1054200091816AE070E00E94BF36F301EB55FE4FB8
:105430007183608380914D0290914E028B01081B15
:10544000190B80914B0290914C02C81AD90A2091F5
:105450000801215045EE54E1B801C6010E948F13A6
:105460008091E1048111C9C04C2DDF8ECE8E602F5A
:1054700019A308A3BAA2F8E0FBA38E189F08E82C92
:105480009F8A8E8A2EA13FA1221A330A022D398EBD
:10549000288EBA8EBB8EFF88198D20E130E15F8D9A
:1054A00079A180E198E00E94D81381110E94B31580
:1054B0008091AF048823C1F12091490230914A02C2
:1054C0008091470290914802281B390B8091450238
:1054D000909146020A974091430250914402841BE6
:1054E000950BE82E9A838983022F3C832B8334E229
:1054F0003D83BE82FA801C8124E230E14E8D5F8DB7
:1055000068A179A18AA19BA10E94D813882361F088
:1055100087E598E10E947C13ACA1BDA11C92A092EA
:10552000CA04B2E3B093DD048091E004882309F457
:1055300064C0F0E48F2EF2E09F2ED12CC12CF40138
:1055400081914F01882309F450C0F601E65CFD4FBC
:105550002081318180914D0290914E02281B390BA0
:10556000F601EC5CFD4F8081918140914B0250919E
:105570004C02841B950BE82E9A838983022F3C836F
:105580002B83F8E0FD83E3E02E2E2E82FA801C812F
:1055900028E033E04E8D5F8D68A179A18AA19BA19F
:1055A0000E94D813882309F187E598E10E947C13B3
:1055B000ACA1BDA11C92F40131971082A092C80445
:1055C000F601E25DFD4F808191819093AA04809362
:1055D000A904F601E85DFD4F808191819093A804B4
:1055E0008093A704B2E3B093DD04E2E0CE0ED11CB9
:1055F000F6E0CF16D10409F0A2CF2CA13DA12F5F78
:105600003F4F3DA32CA332E0630E711C46E06416AD
:10561000710409F0DACE8091490290914A022091FA
:10562000470230914802821B930B20914502309132
:1056300046024091430250914402241B350B3F8F98
:105640002E8F99A388A380E18AA38BA38091C401A4
:10565000882309F44AC00091C2011091C3010C5F74
:105660001F4FA0904D02B0904E02C090C001D0904C
:10567000C10154E0C50ED11C80914B0290914C02A7
:10568000C81AD90A60910801600F712F711D6A193B
:105690007B0920E04BEA57E1C6010E949C134C2D88
:1056A000DA82C9820A191B09602F1C830B8388E0E8
:1056B0008D838E83EE8CFF8C08A119A12AA13BA1BA
:1056C0005A817C8198E00E94D813882371F010924F
:1056D000C40187E195E10E947C1381E08093E2019F
:1056E00090ED9093E3048093E2048091BF018823BE
:1056F00009F44BC00091BD011091BE010C5F1F4F1A
:10570000A0904D02B0904E02C090BB01D090BC0161
:1057100064E0C60ED11C80914B0290914C02C81AD5
:10572000D90A60910801600F712F711D6A197B09F8
:1057300020E045EB57E1C6010E949C134C2DDA8214
:10574000C9820A191B09602F1C830B8388E08D8393
:105750008E83EE8CFF8C08A119A12AA13BA15A814E
:105760007C8198E00E94D813882379F01092BF01C1
:1057700087E195E10E947C1381E08093E50180ED53
:105780008093E30482E08093E2048091BA0188234D
:1057900009F44DC00091B8011091B9010C5F1F4F81
:1057A000A0904D02B0904E02C090B601D090B701CB
:1057B00074E0C70ED11C80914B0290914C02C81A24
:1057C000D90A60910801600F712F711D6A197B0958
:1057D00020E049EC57E1C6010E949C134C2DDA826F
:1057E000C9820A191B09602F1C830B8388E08D83F3
:1057F0008E83EE8CFF8C08A119A12AA13BA15A81AE
:105800007C8198E00E94D813882389F01092BA0115
:1058100087E195E10E947C1381E08093270210923A
:10582000E00480ED8093E30483E08093E2048091C0
:10583000B501882309F469C00091B3011091B40146
:105840000C5F1F4FA0904D02B0904E02C090B1016E
:10585000D090B20194E0C90ED11C80914B0290917E
:105860004C02C81AD90A60910801600F712F711D8E
:105870006A197B0920E04FEB57E1C6010E949C1397
:105880004C2DDF8ACE8A0A191B09602F198F088FC9
:1058900088E08A8F8B8F2091490230914A02809153
:1058A000470290914802281B390B80914502909144
:1058B0004602E0914302F09144028E1B9F0BE82EBA
:1058C0009A838983022F3C832B8380E18D838E838F
:1058D000FA801C8120E130E15F89798D88E098E0D1
:1058E0000E94D813882389F01092B50187E195E1D1
:1058F0000E947C1381E08093E0041092270280EDE7
:105900008093E30485E08093E20420902702222024
:1059100059F18091E104811127C02091AF04609179
:10592000490270914A028091470290914802681B97
:10593000790B8091450290914602E0914302F091EB
:10594000440230910E01332311F40C94BF35211120
:10595000B7C20997EE24E3940DEC15E14DEE55E145
:105960008E1B9F0B0E94190D3090E004332009F428
:105970007AC08091E104811126C080914502909106
:105980004602E0914302F091440260914902709115
:105990004A02695F7F4F2091470230914802621BA3
:1059A000730B20910E01222311F40C94CB35059634
:1059B000EE24E39401E316E120E041E456E18E1B7E
:1059C0009F0B0E94190D50E4A52E52E0B52E6EE0FB
:1059D000C62E62E0D62E10E000E07AE0872E912CF1
:1059E000D5018D915D018823A9F1F801E25DFD4F9C
:1059F00080819181B4010E94BF369B01F801EC5C6B
:105A0000FD4F71836083F801E85DFD4F80819181D6
:105A1000B4010E94BF36F801E65CFD4F71836083DC
:105A20006350710980914D0290914E02681B790B71
:105A3000C901039720914B0230914C02821B930BBA
:105A4000F6012081222309F458C220E04DE556E1F9
:105A50000E948F13FFEFCF1ADF0A0E5F1F4F063031
:105A6000110509F0BDCF8091DE049091DF04181676
:105A70001906C4F5A0904F02B090500260904D02FC
:105A800070904E02C501409600910801080F192F31
:105A9000111D06191709C0905102D0905202809032
:105AA0004B0290904C02C601809620E045EE56E1F4
:105AB000B801881999090E948F13B50166197709F1
:105AC00020E047E656E1C601881999090E948F1324
:105AD000C601409720E045EE56E1B80188199909C2
:105AE0000E948F1321ED622E21E0722E35EC832E61
:105AF00031E0932E25E02EA34AE0E42EF12CA8AD50
:105B0000B9ADAD90BD90B9AFA8AF1A141B040CF09D
:105B10007CC0ECA9FDA980819181B7010E94BF36AC
:105B20006B01D3016D937C93EAA9FBA980819181DC
:105B3000B7010E94BF368B01D4016D937C93B9E20B
:105B4000AB16B104ACF080914D0290914E026350BF
:105B50007109681B790BE0914B02F0914C0220E037
:105B600044E157E1C60103978E1B9F0B0E948F13E0
:105B7000C5014F970A97B0F480914D0290914E0263
:105B8000B80162507109681B790BE0914B02F091EA
:105B90004C0220E04EE057E1C60102978E1B9F0B9E
:105BA0000E948F13C50145970A97B0F480914D026A
:105BB00090914E02B80161507109681B790BE09118
:105BC0004B02F0914C0220E049E057E1C6010197F9
:105BD0008E1B9F0B0E948F13C5010B970A9708F02D
:105BE00090C180914D0290914E02B801681B790BD3
:105BF00080914B0290914C0220E045E057E1F60184
:105C0000E81BF90BCF010E948F133EA131503EA338
:105C10004CA95DA94E5F5F4F5DAB4CAB52E0650E8A
:105C2000711C6AA97BA96E5F7F4F7BAB6AAB72E088
:105C3000870E911C311163CF222049F020E049ECFE
:105C400057E161E070E08AE090E00E949C1333200D
:105C500049F020E04FEB57E161E070E08AE090E02E
:105C60000E949C138091E501882349F020E045EBD8
:105C700057E161E070E083E190E00E949C13809125
:105C8000E201882349F020E04BEA57E161E070E04F
:105C90008CE190E00E949C131C821B828BE491E0BB
:105CA0009A83898385E095E09F838E8380E890E0E6
:105CB0009987888780E490E09B878A8785E08D8B31
:105CC00081E08C8B1F861E86198A188A1D861C8689
:105CD00081E090E09B8B8A8B1D828091E304882376
:105CE00019F18091E204813009F023C184E190E050
:105CF0009F878E879D878C87998B888B60EA77E159
:105D0000CE0101960E94A11285E090E09F878E87C8
:105D10009D878C878EE190E0998B888B6EE877E188
:105D2000CE0101960E94A11201E010E0CC24C394A0
:105D3000D12C40E0B601C8010E943B148FEFC81A75
:105D4000D80A99E0C916D104A1F70F5F1F4F093097
:105D5000110561F768E081E090E00E94591483E04A
:105D600090E09F878E879D878C87998B888B409149
:105D7000050150E070E060E02AE0CE0101960E944B
:105D8000691B04E610E0CC24C394D12C40E0B6019A
:105D9000C8010E943B14AFEFCA1ADA0AB9E0CB1669
:105DA000D104A1F70F5F1F4F0F37110561F76BE1AA
:105DB00084E690E00E94591486E690E09F878E87E3
:105DC0009D878C8783E090E0998B888B6091DE01C2
:105DD0007091DF01CE0101960E94BD1B8091DD0113
:105DE00081110E94C3130E9438140C941122209137
:105DF00008012150B501681B790B48E552E1C60145
:105E00002AC0B501681B790BEE24E39406E112E188
:105E100020E046E352E1C6018A1B9B0B0E94190D4C
:105E200057C9B501681B790BEE24E39404ED11E129
:105E300020E044EF51E1EFCF209107012150B5015F
:105E4000681B790BC30134E0880F991F3A95E1F77D
:105E5000079648EA51E18A1B9B0B0E948F1338C9B1
:105E600068A579A5681B790B20E046E951E1C7CF09
:105E7000209107012150B501681B790BC30104E093
:105E8000880F991F0A95E1F7039648E551E1E3CFA2
:105E9000B501681B790B20E046E351E1B0CFB501B5
:105EA000681B790B20E044E251E1A9CFB401681BE3
:105EB000790B20E042E151E1A2CFC60102967AC9F6
:105EC000233048F0079620E047EA55E18E1B9F0BF0
:105ED0000E948F1349CD409620E04DE955E1F6CF61
:105EE0000A978E1B9F0B233020F020E045E355E1FD
:105EF000EFCF20E04DE955E1EBCF20E043E556E15F
:105F0000A7CDFBE0AF16B1040CF07FCE80914D021F
:105F100090914E02B801681B790B80914B029091D1
:105F20004C0241E09601281B390BC9010E943B1429
:105F30006CCE8230D9F484E190E09F878E879D8774
:105F40008C87998B888B6CE777E1CE0101960E9454
:105F5000A11289E190E09F878E879D878C878EE1D3
:105F600090E0998B888B60E777E1DACE8330D9F4C3
:105F700088E290E09F878E879D878C8704E110E000
:105F8000198B088B64E677E1CE0101960E94A1127D
:105F90001F870E871D870C878EE190E0998B888B79
:105FA00062E577E1BDCE8530E9F488E290E09F8735
:105FB0008E879D878C8784E190E0998B888B68E43D
:105FC00077E1CE0101960E94A1128FE090E09F87B9
:105FD0008E879D878C878EE190E0998B888B67E315
:105FE00077E19ECE843009F09FCE01E410E01F8758
:105FF0000E871D870C878AE090E0998B888B60E381
:1060000077E1CE0101960E94A11287E390E09F877D
:106010008E879D878C878FE090E0998B888B64E2D8
:1060200077E1CE0101960E94A1121F870E871D877E
:106030000C8784E190E0998B888B6BE177E170CEDF
:10604000413852405CF04091AD045091AE0480580C
:1060500092404817590714F40C9467278091AB04B9
:106060009091AC044091000250910102840F951F61
:1060700097FF02C00C947C279093AC048093AB04F0
:106080008091FF01882311F40C9486278091FE01F2
:1060900081110C94862710920102109200022111A6
:1060A00015C08DE498E10E947C1381E08093CB04BD
:1060B0008091DD04811103C08FE08093DD04809125
:1060C000DC04811103C08AE08093DC0481E08093CA
:1060D000FD011092FC018091FA019091FB01AC014D
:1060E0004F5951092091AB043091AC042417350766
:1060F000BCF0805A91099093AC048093AB04109249
:106100000102109200028091FD01811104C08DE412
:1061100098E10E947C1381E08093FD011092FC01C4
:106120000091AB041091AC04013441E0140774F009
:1061300080E10E942314882349F080E80E94231400
:10614000882321F01093F9010093F8018091FE015A
:10615000811119C08091FC01811115C080E10E945C
:106160002314013451E0150774F4882361F080E8AA
:106170000E942314882339F0C80180569F4F9093C2
:10618000F9018093F80180910C0190910D0120910B
:10619000F6013091F701821B930B2091AD043091F1
:1061A000AE04820F931F2AE030E0B9010E94BF368F
:1061B000709346026093450280910A0190910B0111
:1061C0004091F4015091F501841B950B800F911FB4
:1061D000B9010E94BF3670934A02609349028091D0
:1061E000E004882309F44EC080900C0290900D02C8
:1061F000E0E4F2E068E2C62E62E0D62E2EE232E063
:106200000EE012E073E4A72E72E0B72E48E1808121
:10621000882369F1D9018D919C91D8015C91552316
:1062200011F40C948D278096D90111969C938E932E
:106230008D919C9197FD1082881699060CF410821E
:10624000B2010E94BF363B01D6018D919C91B201F3
:106250000E94BF36469DD001479DB00D1124AE5916
:10626000BD4FA60FB71F8C91853108F01082319673
:10627000B2E0CB0ED11C2E5F3F4F0F5F1F4FAE160B
:10628000BF0629F6E0E2F2E0FFA3EEA307E112E089
:10629000EDE1F2E041E1A42E42E0B42E50E2252EE1
:1062A00052E0352E48E1FF24F394D1018D911D0178
:1062B000882309F446C0D8012D913C91D501CD9099
:1062C000DC90C601805B9F4FB2010E94BF363B014C
:1062D0008081B60166557F4F6B01882311F40C94C1
:1062E0009027C90186559F4FB2010E94BF364B01CE
:1062F000469FC001479F900D11248E599D4F680EF7
:10630000791ED3018C91853108F01082C601B2014B
:106310000E94BF36489DD001499DB00D1124AE5951
:10632000BD4FA60FB71F8C91853108F41082808174
:10633000882311F40C94B9272B5F3F4FD8012D937C
:106340003C930E5F1F4F3196B2E0AB0EB11C23E2BF
:10635000221622E0320609F0A8CF4FE552E05DA3F5
:106360004CA309E5C02E02E0D02E83E2A82E82E0E5
:10637000B82E03E512E092E6292E92E0392E4A016A
:1063800023E0622E712C38E1F32EEE24E394D40145
:106390008D914D01882309F45DC0D601ED91FC91EA
:1063A000D8018D919C91805B9F4FB2010E94BF36B6
:1063B0009B01D5018C91882311F40C94BD27CF014A
:1063C00086559F4FB2010E94BF36F69EF001F79EA0
:1063D000F00D1124EE59FD4FE20FF31F808185313E
:1063E00010F0F50110820E943636B3010E94BF36CC
:1063F000F601208131818130910511F00C94D42770
:10640000D801ED91FC913A97C901805B9F4FB20191
:106410000E94BF369B01CF01B2010E94BF36F29E9F
:10642000D001F39EB00D1124AE59BD4FA60FB71F7A
:106430008C91853118F4D801ED93FC93F60180819D
:106440009181D5012C91222311F40C94F927059602
:1064500091838083F2E0CF0ED11C2FEFA21AB20AF3
:106460000E5F1F4F2814390409F091CF8091DE048C
:106470009091DF04181619060CF07BC18091A204DC
:106480009091A30480569F4FB2010E94BF368B01AA
:106490002091A4043091A5048091A604882311F4CE
:1064A0000C94FC27C901865B9E4FB2010E94BF3647
:1064B00088E1869FF001879FF00D1124EE59FD4F72
:1064C000E00FF11F8081853110F01092A6048091B9
:1064D000A604882311F40C9415282E5F3F4F3093A7
:1064E000A5042093A4040E94363664E670E00E945E
:1064F000BF369C010091A2041091A3048091A404D2
:106500009091A504232BE9F4A80140515109EFE52E
:10651000F2E030E020E061E0719171110DC0DF0127
:1065200011976C93D901A75ABD4F8D939C93D901B4
:10653000AD5ABD4F4D935C932E5F3F4F26303105D2
:1065400059F72AE030E0B9010E94BF36FB01709391
:10655000520260935102C801B9010E94BF36709384
:10656000500260934F0280914D0290914E029B0128
:10657000281B390BCF01409740914B0250914C02A0
:10658000841B950B482F9F8F8E8F622F39A328A3D2
:106590008EE38AA381E28BA32091490230914A02C3
:1065A0008091470290914802281B390B8091450247
:1065B00090914602E0914302F09144028E1B9F0BA2
:1065C000E82E9F8B8E8B022F398F288F80E18A8F48
:1065D0008B8FFF88198D20E130E15F8D79A18EE3EB
:1065E00091E20E94D81381110E94B315B0E4AB2E42
:1065F000B2E0BB2ED12CC12C18E0912E88248394BC
:10660000D5018D915D01882309F456C0F601E65C41
:10661000FD4F2081318180914D0290914E02281BC7
:10662000390BF601EC5CFD4F8081918140914B026A
:1066300050914C02841B950BE82E9A838983022F7C
:106640003C832B839D82B3E0BE83FA801C8128E0CB
:1066500033E04E8D5F8D68A179A18AA19BA10E9434
:10666000D813882349F187E598E10E947C13809133
:10667000DE049091DF0401979093DF048093DE04A1
:106680000E94EC15F501319710828092C804F60142
:10669000E25DFD4F808191819093AA048093A904CB
:1066A000F601E85DFD4F808191819093A80480936D
:1066B000A704E2E3E093DD04F2E0CF0ED11C26E074
:1066C000C216D10409F09CCF8091AF04882309F44D
:1066D00047C080912702882309F442C020914902D3
:1066E00030914A028091470290914802281B390B51
:1066F00080914502909146020A9740914302509141
:106700004402841B950BE82E9A838983022F3C83D5
:106710002B8384E28D8380E18E83FA801C8124E2C6
:1067200030E14E8D5F8D68A179A18AA19BA10E9465
:10673000D8138823A9F087E598E10E947C13809103
:10674000DE049091DF0401979093DF048093DE04D0
:106750000E94EC1581E08093CA0432E33093DD049B
:106760008091DE049091DF04892B19F484E68093F4
:1067700026028091DD04882309F463C01091CB04C4
:106780008091AD049091AE04805B9F4F2091AB044B
:106790003091AC04390140EA640E711C0091CA04C6
:1067A000205B3F4FF090C904E090C804C090A9045A
:1067B000D090AA04A090A704B090A8044CEC54E098
:1067C0006CEB74E079A768A7E0EBF4E066ED74E0A9
:1067D000DA018D909D90AD01892851F54D01B2E00F
:1067E0008B1A9108A2E32A2E312CD4012D923C92CF
:1067F000112331F0A8A5B9A58D939C937182608275
:10680000002331F0A8A5B9A58D939C9331832083F3
:10681000FF2031F0A8A5B9A58D939C9331832083E7
:10682000EE2031F0A8A5B9A5CD92DC92B182A0826C
:10683000A8A5B9A51296B9A7A8A732966417750797
:1068400039F68091DC04882311F40C9419280E94F5
:10685000363664E070E00E94BF3628E0E1E2F1E005
:10686000DE01569601900D922A95E1F728E0E9E2C3
:10687000F1E0DE01119601900D922A95E1F7209149
:10688000AF04211101C00496FE01E80FF91F4689EB
:106890002091DA043091DB04240F311D47FD3A9535
:1068A0003093DB042093DA04E1E0F0E0EC0FFD1F0D
:1068B0008E0F9F1FDC012C918091D8049091D904F8
:1068C000820F911D27FD9A959093D9048093D80447
:1068D000ECECF4E0F9AFE8AF20EB34E03BAB2AABF3
:1068E0004CEB54E05DAB4CAB76ED872E74E0972E0D
:1068F0006A0159018F01D8018D919C9118161906D2
:106900000CF06BC00E94363664E070E00E94BF3627
:106910002091CB04222381F0EAE0F0E0F9ABE8AB70
:1069200025E030E03FA72EA74FE050E05DA74CA741
:106930006FE070E07BA76AA72091CA04222381F050
:10694000A4E1B0E0B9ABA8ABE4E1F0E0FFA7EEA7AB
:1069500024E130E03DA72CA744E150E05BA74AA723
:106960002091C904222381F062E370E079AB68AB27
:10697000A2E3B0E0BFA7AEA7E2E3F0E0FDA7ECA77B
:1069800022E330E03BA72AA72091C804222381F00C
:106990004AE050E059AB48AB6AE070E07FA76EA7D1
:1069A000AAE0B0E0BDA7ACA7EAE0F0E0FBA7EAA749
:1069B000009711F00C942328D6018D919C9111978A
:1069C0002AA43BA4820D931D8D939C93D8018D9195
:1069D0009C91119701978D939C930E5F1F4FB2E08E
:1069E000AB0EB11CE2E0CE0ED11C8016910609F070
:1069F00082CF1092CB041092CA041092C904109254
:106A0000C8048091E104811147C0F0900F0190907B
:106A1000FD01F11006C080910801692D70E08230FF
:106A200011F070E060E0C0904902D0904A022091DD
:106A30004702309148026C0D7D1D621B730B009163
:106A4000450210914602A0904302B0904402C80152
:106A50008A199B09FBE0CF0ED11CC21AD30A2091E0
:106A60000E01222311F40C94462820E040EF50E15F
:106A70000E949C13C801992009F479C003968A19D1
:106A80009B0921E0F11003C020910801215040ED45
:106A900050E1B6010E949C1342E6242E42E0342EBF
:106AA00056E0852E912C68E1F62E540126E0A21ABC
:106AB000B108A4014E5F5F4F59A748A7D12CC12C44
:106AC000712C612CA0914B02B0914C02CD010F971B
:106AD000C816D90614F40C94682882569F4F8C155A
:106AE0009D0514F40C94682880914D0290914E02FB
:106AF0009C012F503109A216B30614F40C94682897
:106B0000225A3F4F2A153B0514F40C946828F69C32
:106B1000F001F79CF00D1124E20DF31D2081E9EF47
:106B2000E20FED3110F00C946828F0E0E656FA4CD4
:106B30000C94D336F72E012F112F682868281C2FAC
:106B4000302F382F482F4F2F562F68286828682855
:106B50005D285D285D285D285D285D285D285D280D
:106B60005D285D285D285D285D285D285D280496E8
:106B700020E046EC50E1B6018A199B098BCF211128
:106B8000AFC90996EE24E3940BE515E120E04BE74D
:106B900055E10C94B02C0597EE24E3940FE016E138
:106BA00020E04FE156E10C94DF2C992311F40C9472
:106BB00058250C944C26109201021092000281E09C
:106BC0008093FC011092FE0185E298E10E947C1303
:106BD0000C9458258F929F92AF92BF92CF92DF92E2
:106BE000EF92FF92CF93DF93EC01688179818A81E4
:106BF0009B81611571058105910521F464E279EDB0
:106C00008BE597E02DE133EF41E050E00E945C36E8
:106C100049015A019B01AC01A7EAB1E40E947B360D
:106C20006B017C01ACEEB4EFA50194010E948936A2
:106C3000DC01CB018C0D9D1DAE1DBF1DB7FF03C038
:106C40000197A109B04888839983AA83BB839F7762
:106C5000DF91CF91FF90EF90DF90CF90BF90AF90FA
:106C60009F908F9008950E94EA3508958DE191E0FC
:106C70000E94EA350895B0E0A0E080931D01909352
:106C80001E01A0931F01B09320010895F999FECF32
:106C900092BD81BDF89A992780B50895262FF9995C
:106CA000FECF1FBA92BD81BD20BD0FB6F894FA9AEF
:106CB000F99A0FBE01960895052E97FB1EF40094D5
:106CC0000E94733657FD07D00E948E3607FC03D012
:106CD0004EF40C94733650954095309521953F4F66
:106CE0004F4F5F4F089590958095709561957F4FB8
:106CF0008F4F9F4F08950E94B036A59F900DB49F6F
:106D0000900DA49F800D911D11240895B7FF0C9440
:106D10007B360E947B36821B930B0895A1E21A2ECC
:106D2000AA1BBB1BFD010DC0AA1FBB1FEE1FFF1F2F
:106D3000A217B307E407F50720F0A21BB30BE40B7F
:106D4000F50B661F771F881F991F1A9469F76095C6
:106D50007095809590959B01AC01BD01CF01089580
:106D6000A29FB001B39FC001A39F700D811D11248C
:106D7000911DB29F700D811D1124911D089597FBE7
:106D8000072E16F4009407D077FD09D00E94D9365B
:106D900007FC05D03EF4909581959F4F089570951E
:106DA00061957F4F0895EE0FFF1F0590F491E02D40
:106DB0000994AA1BBB1B51E107C0AA1FBB1FA61742
:106DC000B70710F0A61BB70B881F991F5A95A9F794
:0E6DD00080959095BC01CD010895F894FFCFF9
:106DDE0002000400100301010101360180020101CD
:106DEE0001FFFFFFFF00E1000000000000010000B6
:106DFE000007F9000001FF0000000003FD00000382
:106E0E00F69D091F09C2083808AB07540735050857
:106E1E0005B104E002AC0000000000F6115B116643
:106E2E001B651B00C18081000000000000006B0F7D
:106E3E00D6108C0F810FD20F900FAE0F00000000F6
:086E4E0092145B11661B651B29
:00000001FF
